:1066990001190000090101240200000301FA0400A4
:1066A900FA0500030A0A5A0B001E0C00FA0D000332
:1066B9000E00040F0164100096120132130AFA1435
:1066C900010215000217010A1801FA1905321A0107
:1066D9000A1B01FA1C05321FFFFF20FFFF23011EC1
:1066E9002400642A00FA2B00FA2C50782D003D2E44
:1066F90000462F001E3000643250783300003432D7
:10670900FA350164360164370150380A643C006483
:106719003E003C3F000140FFFF411450420A5A43EA
:106729000AC84405324500B44600FA470148480200
:10673900034C00FA4EFFFF500606510596520A32E5
:10674900530B46540A9656020257054658000259F9
:106759000A465A32FA5B010A5C0A325E000A5F0095
:10676900FE61FFFF64021066000267FFFF6A0A3CD0
:106779006B00006C32967300007400007801327966
:1067890001327E00FE81FFFF84FFFF8500AF860096
:10679900018700FA89010A8A00009900009D0A967A
:1067A9009E00019FFFFFA0FFFFFAFAFA0065006F44
:1067B90000790083008D009700A100AC00B600C0ED
:1067C90000CA00D400DE00E800F20058006000684A
:1067D90000700078008000880090009800A000A850
:1067E90000B000B800C100C800D000D800DF00E642
:1067F90000EE00F600410047004D00530059005FCC
:106809000065006C00710077007D00830089008FAE
:106819000095009B00A200A700AC00B200B900C01F
:1068290000C500CA00D200D500DD00E100E700EF95
:103A39009007C5E0FEA3E0FF90669B126972E493CC
:103A4900F599906699E493FC740193FDEFB5050728
:103A5900EEB50403754D009007C51269592275A783
:103A69001085F97385FA747E017F00E57412694B3C
:103A7900E5732FFF50010E8E5A8F5B900017E0FC03
:103A8900A3E0FDEF2DFDEE3CFC8C5C8D5D2275A75E
:103A99001085F97385FA747E017F00E57412694B0C
:103AA900E5732FFF50010E8E5A8F5BAC2CAD2DEFB5
:103AB9002DFDEE3CFC8C5C8D5D22E55DF5FBE55C46
:103AC900F5FCD29322E55DF5E9E55CF5EAD29422AD
:103AD900E55DF5EBE55CF5ECD29122E55DF5EDE50B
:103AE9005CF5EED29222E55DF5FDE55CF5FED28747
:103AF90022E55DF5CEE55CF5CFD29022AE5AAF5BFB
:103B0900740A8E048F05FF12693B8C5C8D5DAE5A79
:103B1900AF5B740A8E048F05FF1269668C5A8D5B40
:103B2900E55B455A6013740AC3955BFFE4955AFE39
:103B39008E5A8F5B785C12699FE573A85CB8001593
:103B4900D3955D4010E573C3955DFFE4955CFE8EEA
:103B59005C8F5D8010E5732424C3955DFFE4955C5B
:103B6900FE8E5C8F5DAE5CAF5D74236F4E60067434
:103B7900246F4E701AAE5CAF5D74236F4E7005757D
:103B890073018003757302755D22755C008003758E
:103B9900730022900095E0B40104C2108002D21093
:103BA900900096E0B40104C2118002D2119000D3B2
:103BB900E075F0DCA4FFAEF0740A8E048F05FF12E5
:103BC900693B9007BBECF0A3EDF0A20D401674031E
:103BD9008C068D0712694B74011200399007B9EEF2
:103BE900F0A3EFF07E017F00900091E012694B9005
:103BF90000D4E08E048F05FF12693B740AFF126935
:103C09003B8D609000DDE075F0DCA4FFAEF0740A36
:103C19008E048F05FF12693B9007BFECF0A3EDF00E
:103C29009000DFE060139000DFE0F5F0741684FF88
:103C39007E00EF9007CDF0800674649007CDF09078
:103C490000D5E0900079F090011FE0900063F090BA
:103C590000AEE0900065F09000D7E0900066F0902B
:103C69000083E0900067F0900109E090006CF0900B
:103C7900016DE090006DF090016EE090006EF090A3
:103C8900016FE090006FF0A22AB3401690016DE039
:103C9900700C90016EE0700690016FE06002800286
:103CA900C22A74E3900078F09000BEE0B40B087467
:103CB900E3900078F0805A9000BEE0B419129000A9
:103CC900D4E09067A012008CE493900078F08041D2
:103CD9009000BEE0B41E129000D4E09067BE1200BE
:103CE9008CE493900078F080289000BEE0B428120C
:103CF9009000D4E09067E812008CE493900078F08B
:103D0900800F9000BEE0B446089000B5E0900078BE
:103D1900F09000EEE0FE9000BCE06E600A9000BCFE
:103D2900E09000EEF0D22990007CE0FE9000BBE02C
:103D3900B5063390007EE0FE9000D9E0B5062790E5
:103D4900007DE0FE9000E7E0B5061B900080E0FEF4
:103D590090008EE0B5060F90007FE0FE9000C9E06C
:103D69006E7003023F20900054E0C394055008741C
:103D79000290010AF0801C9000C9E064036006907B
:103D890000E7E06008740790010AF08006740A9061
:103D9900010AF090008EE0B4010674009000F4F07E
:103DA90090008EE0B4020674009000D9F090008E65
:103DB900E0B4030674009000E6F09000BBE06014E4
:103DC90074189000A2F074009006CFF07400900669
:103DD900D0F0800C74009000A2F074189006CFF017
:103DE9009000D9E0D394014014741990010CF07437
:103DF900009006D3F074009006D4F0800C74009003
:103E0900010CF074199006D3F09000C9E0B40308CE
:103E19009000E7E064026002800674009000E7F019
:103E29009000E7E0B401089000C9E06403600280F3
:103E39001A741A90010DF074009000A3F0740090A8
:103E490006D7F074009006D8F080339000BBE0B438
:103E5900021A741A9000A3F0740090010DF0740016
:103E69009006D7F074009006D8F080127400900084
:103E7900A3F0740090010DF0741A9006D7F0900029
:103E8900C9E0B402069000E7E0600280147404906F
:103E990006E3F074059006E7F074069006EBF080EF
:103EA9002474009006E3F074009006E4F074009026
:103EB90006E7F074009006E8F074009006EBF074E1
:103EC900009006ECF0D2299000BBE090007CF090C5
:103ED90000E7E090007DF09000D9E090007EF0903E
:103EE90000C9E090007FF090008EE0900080F09093
:103EF900008EE0900064F09000C9E0900068F090B6
:103F090000E7E0900069F09000BBE090006AF09053
:103F190000D9E090006BF09000F1E0B40117900037
:103F290023740FF0A374FFF0900025E4F0A3F0745C
:103F3900029000F1F09000F1E0B40341900025E017
:103F4900FEA3E0FF900023E0FCA3E0FD1269977453
:103F59001012694B7408120039EF900075F0EF7078
:103F69000674FF900075F074009000F1F090002441
:103F7900E0900076F0900023E0900077F0900082C6
:103F8900E0900043F0900043E0240C900044F0904E
:103F99000043E02418900045F0900044E0D39424B5
:103FA900400B900044E0C39424900044F0900045F5
:103FB900E0D39424400B900045E0C394249000453D
:103FC900F0900049E4F0900043E06423600790001A
:103FD90043E0B42420900043E0B423067402900027
:103FE90049F0900043E0B424069000497401F09030
:103FF90000437401F090004AE4F0900044E0642327
:104009006007900044E0B42420900044E0B4230603
:10401900740290004AF0900044E0B4240690004AEB
:104029007401F09000447401F090004BE4F09000AA
:1040390045E064236007900045E0B42420900045E2
:10404900E0B42306740290004BF0900045E0B424DC
:104059000690004B7401F09000457401F0900082C5
:10406900E0FE9000E5E02E90004DF09000C0E0B435
:10407900016390004DE06412600790004DE0B424A4
:104089000690004DE004F090004DE0641160079047
:10409900004DE0B4230690004DE014F090004DE08F
:1040A900D39424400B90004DE0C3942490004DF02C
:1040B90090004DE0D39412400D90004DE0C394124E
:1040C90090004EF0800A90004DE0241290004EF0CE
:1040D900755112807990004DE0640C600F90004D8D
:1040E900E0641A600790004DE0B4240690004DE0AA
:1040F90004F090004DE0640B600F90004DE06419EE
:10410900600790004DE0B4230690004DE014F09054
:10411900004DE0D39424400B90004DE0C3942490CB
:10412900004DF090004DE0D3940C400B90004DE011
:10413900C3940C90004DF090004DE0D3940C400BCB
:1041490090004DE0C3940C90004DF075510C900017
:10415900C8E0900046F0900046E075F00C84AFF09E
:104169007E00EF4E7006900046E004F0900046E0B5
:104179000475F00C84AFF07E00EF4E700690004697
:10418900E014F0900046E0B449069000467401F04E
:10419900900046E0D39424400F900046E0C3942455
:1041A900900046F0D2238002C223900046E0240CFE
:1041B900900047F0900046E02418900048F09000E5
:1041C90047E0D39424400B900047E0C39424900027
:1041D90047F0900048E0D39424400B900048E0C396
:1041E9009424900048F022C293C294C291C292C210
:1041F90087C290E5B554EFF5B5E5B554DFF5B5C21D
:1042090096C295C2A0C297C2A2C2A1E5B554BFF594
:10421900B5E5B5547FF5B5E5B554FBF5B5C21275ED
:104229005E469000CBE07005756D028003756D03E5
:1042390075550075540090000C74FFF0A374DCF000
:10424900C218C21AC21C74C8900037F074C8900012
:104259003BF074C890003FF0755300755200C20DD1
:10426900754600E56FB40903756F0075630090002A
:1042790019E4F0A3F0757010C215C216C2179007A1
:10428900BBE0FEA3E0FF740312694B74011200390D
:104299009007B9EEF0A3EFF0C2027557007556000A
:1042A900900010E4F0A3F0C22B75590075580090E6
:1042B900008DE075F032A4FDACF0900021ECF0A384
:1042C900EDF0C23BA22FB39205A230B39206A23100
:1042D900B39207A232B39208A233B39209A234B3BC
:1042E900920AA235B3920BA236B3920C2275A7108B
:1042F90085F97385FA747E017F00E57412694BE5CF
:10430900732FFF50010E8E5A8F5BAC5CAD5DEF2DA4
:10431900FDEE3CFC8C5C8D5D123AC3123ACE123A2A
:10432900D99000C9E0B40309123AE4123AEF123AFB
:10433900FA75A7002285F97385FA747E017F00E575
:104349007412694BE5732FFF50010E8E5A8F5B7EF5
:10435900017F76900106E012694BAC5AAD5BED2FF7
:10436900FFEC3EFE8E5C8F5DE55DF5EDE55CF5EEFF
:10437900900079E4F07412900050F02285F9738569
:10438900FA747E017F00E57412694BE5732FFF50C3
:10439900010E8E5A8F5B9007BBE0FCA3E0FDEF2D69
:1043A900FDEE3CFC8C5C8D5DE55DF5FDE55CF5FEA7
:1043B90022056422A2DBB340089000D5E090007981
:1043C900F0A2DCB34006C296C295C2A075D84022BD
:1043D90085A77275A7109000C9E064036007900073
:1043E900E7E0B4022CA2D8B34002C293A2D9B340E9
:1043F90002C294A2DAB34002C291A2DBB34002C264
:1044090092A2DCB34002C287A2DDB34002C290800F
:104419002DA2D8B3400AC2939000E7E06002C2928D
:10442900A2D9B3400AC2949000E7E06002C287A211
:10443900DAB3400AC2919000E7E06002C29075D8F1
:10444900408572A722900047E4936406600280FECB
:1044590074C89007C1F8E4F0E8A3F075B500758455
:104469000175A70075FFA090004CE4F075C910759F
:10447900A70F75A1C775A70075D90075CE0C75A7CB
:104489000F75F1FE75F2FF75F30775F47875A4BA27
:1044990075A5FF75A60775AE0075AFFF75D4817553
:1044A900D5FF75D6FF75D7FF75A70075A20175A150
:1044B9004775F80975D80075D90475DD0975DE09E0
:1044C90075D84075A71075D80075D90475DA0975BE
:1044D900DB0975DC0975DD0975DE0975DF0975D834
:1044E9004075A70075E60875E71075BC0175BE042F
:1044F90075BD6C75BE0775BDA075BE0875BD017526
:10450900BC0075BB1875BC2075BA0875E88075D1F3
:104519001375A70F75E10575E20075C7401241F0E3
:10452900759700759780740A12692B7597C0E5977E
:104539005420700280F8758F0275A700D2AF759864
:104549000075A90C75A70F75AB4375ADFB75AC1E4E
:1045590075A71075C91875CA0075CB0075C804759B
:10456900A700758912758E04758C00758A00C2A919
:10457900D28C758D00758B00D2ABD28E75EF067516
:10458900D944C2997509C87508001200E975B500C2
:104599001204E974639007C1F8E4F0E8A3F0120388
:1045A9007574C89007C1F8E4F0E8A3F0750964755B
:1045B90008001200E9900064E090008EF090008EEF
:1045C900E0D39403400C740090008EF074009000C6
:1045D90064F0C22090008EE09062AAF828287380C7
:1045E90028A2B44002D220802075A70F75F30F7559
:1045F900A700A2A34002D220800F75A70F75F31759
:0946090075A700A2A44002D22012
:0C62AA000245E80245EA0245F202460304
:10461200A220B3405E757308E573D3940E501FE574
:10462200739007C1F8E4F0E8A3F01202447509643C
:104632007508001200E97873740126F650DA7402E4
:104642009000CAF0900064E090008EF090008EE03E
:104652009062B6F8282873801674009000F4F080F7
:0F4662000E74009000D9F0800674009000E6F00E
:0C62B60002465902465B02466302466B3A
:10467100D21F805C757301E573D39407501FE573F6
:104681009007C1F8E4F0E8A3F012024475096475DB
:1046910008001200E97873740126F650DA7401906B
:1046A10000CAF0900064E090008EF090008EE090DF
:1046B10062C2F8282873801674009000F4F0800E0E
:0E46C10074009000D9F0800674009000E6F0BE
:0C62C2000246B70246B90246C10246C9B6
:1046CF00C21F900063E090011FF0900064E0900023
:1046DF008EF0900065E09000AEF0900066E09000E4
:1046EF00D7F0900067E0900083F0900068E09000B2
:1046FF00C9F0900069E09000E7F090006AE0900048
:10470F00BBF090006BE09000D9F090006CE090014E
:10471F0009F090006DE090016DF090006EE0900157
:10472F006EF090006FE090016FF090016DE0700CF3
:10473F0090016EE0700690016FE060028004C22A63
:10474F008002D22A9000D4E07006740A9000D4F050
:10475F009000B5E0700674E39000B5F09000BBE0F8
:10476F000490007CF09000BCE09000EEF0123B9CB7
:10477F00E5B54401F5B57406900052F07401900050
:10478F0053F07403900055F07405900056F0743F89
:10479F00900057F07405900058F07401900059F094
:1047AF00740090005EF07400900061F074FF900050
:1047BF0062F07433900158F07436900159F0742DF3
:1047CF0090015AF0743290015BF0742090015CF00C
:1047DF00743690015DF0744390015EF0747990012E
:1047EF005FF0746C900160F07420900161F07420A0
:1047FF00900162F07456900163F07456900164F06A
:10480F007454900165F07420900166F09000F0E010
:10481F00900075F09000A7E0900076F09000A8E06F
:10482F00900077F0A2B6B3920EA2B3B3920FA2A4E8
:10483F00B39226A2B4B39227A2A3B3922890007189
:10484F00E4F0756F00743A900781F074FD90078261
:10485F00F0900072E4F09007BBE0FEA3E0FF74035A
:10486F0012694B74011200399007B9EEF0A3EFF003
:10487F00756E01900050E4F0C225756300C213D22B
:10488F0014C202757100C22DD203C22ED204C22FE0
:10489F00D205C230D206C231D207C232D208C233D9
:1048AF00D209C234D20AC235D20BC236D20CC221BF
:1048BF00C222C223C224C22912009E755F00756BEB
:1048CF000075610075653275660075670075680063
:1048DF00756900756A00900019E4F0A3F0756C001B
:1048EF00D2B2D2A4D2B0D2B1D2A3D2A7D2A6D2A5DD
:1048FF00D2B790008DE0D394FA400674FA90008DF1
:10490F00F07E017F00900077E012694B900076E017
:10491F002FFF50010E900023EEF0A3EFF0EFD39492
:10492F00FFEE940F4007900023E4F0A3F090007582
:10493F00E0700674FF900075F09000CAE0D3940207
:10494F00400674019000CAF09000CBE07005756DC1
:10495F00028003756D039000CCE0D3940140067480
:10496F00009000CCF09000D2E0C3940A5006740A75
:10497F009000D2F09000DCE0700674019000DCF043
:10498F009000DCE0B4FF0674FE9000DCF09000E3D2
:10499F00E0D394FE400674FE9000E3F0900109E02E
:1049AF00D3940240067401900109F090011FE0D3E7
:1049BF0094014006740190011FF074019000E9F01A
:1049CF0074019000EAF074009000F1F07407900108
:1049DF000EF07400900111F074299006C7F0742A3C
:1049EF009006CBF0741B9006DBF0741C9006DFF082
:1049FF00D29C9000BCE0D39404400674049000BC99
:104A0F00F0E570D3941040037570109006C8E0D392
:104A1F00940C400674009006C8F09006CCE0D39436
:104A2F000C400674009006CCF09006D0E0D3940CA6
:104A3F00400674009006D0F09006D4E0D3940C405A
:104A4F000674009006D4F09006D8E0D3940C40067C
:104A5F0074009006D8F09006DCE0D3940C400674F6
:104A6F00009006DCF09006E0E0D3940C4006740052
:104A7F009006E0F09006E4E0D3940C4006740090AA
:104A8F0006E4F09006E8E0D3940C4006740090061C
:104A9F00E8F09006ECE0D3940C400674009006EC1E
:104AAF00F0D2EC75CF01A298B34005C2981206461A
:104ABF00E54D6006A299B3B340028005C299120C6E
:104ACF0057E54E64016005E54EB4040280D5C28EF1
:104ADF007E107F00E56412694BE58D75F010A4FD23
:104AEF00ACF0EF2DFDEE3CFCE58B75F01084FF7EF6
:104AFF0000ED2FFFEC3EFE8E548F55D28E9000AE00
:104B0F00E060099000AEE0C3943D400280569000F3
:104B1F001B12695990001BE0FEA3E0FF90001DE0FF
:104B2F00FCA3E0FDEFB5053CEEB50438B21EA20DB7
:104B3F00B34013A21EB34008E5B54404F5B5800693
:104B4F00E5B554FBF5B590001DE0FEA3E0FF900026
:104B5F001FE0FCA3E0FDEF2DFDEE3CFC90001DECF3
:104B6F00F0A3EDF09000BBE060099000BBE0C394B0
:104B7F00034002807B122D96A20DB3500990007155
:104B8F00E0C3941C400280069000A5E0F545E54582
:104B9F0075F005A4FFAEF09007C3EEF0A3EFF09011
:104BAF000092E0C395614007E55FC39560500790A1
:104BBF0007C3E4F0A3F0AE2EAF2F9007C3E0FCA322
:104BCF00E0FDEFD39DEE9C400AC297E5B554DFF5AB
:104BDF00B58011900071E0C3942A5008D297E5B5C3
:104BEF004420F5B59000BBE0B40205A297B392A1A3
:104BFF009000BBE0B4031C122EB1AE2EAF2F900766
:104C0F00C3E0FCA3E0FDEFD39DEE9C4004D2978060
:104C1F0002C297900096E06009A2B3300F01B3B3C0
:104C2F0040028039A2B3300F01B34031A2B330112B
:104C3F0001B3401C9000C9E0B40306A221B3B340F6
:104C4F000280067404900050F0D221A211B3920F8B
:104C5F00A211B330B301B34004A211920FA2B63028
:104C6F000E01B35003025301A2B6300E01B350032D
:104C7F00025301A2B6301001B35003025143756EB7
:104C8F00009000AEE0B43D13A210B34008E5B55458
:104C9F00FBF5B58006E5B54404F5B5055EA212B384
:104CAF00B35013AE54AF5590000CE0FCA3E0FDEDF4
:104CBF00C39FEC9E4003024E13E56DB4032EA22B4F
:104CCF00B34022E55EB42303756D01E55EC3942303
:104CDF0050069000507401F0E55ED39423400674A3
:104CEF0002900050F0755E01D22B805CE56DB4022E
:104CFF0006756D01755E23E55EB42305755E018053
:104D0F0047900050E07032E55EC394235006900048
:104D1F00507401F0E55ED394234006740290005066
:104D2F00F0E55EC394235002D225E55ED394234071
:104D3F0002D225C296C295C2A09000CBE0B4010565
:104D4F001241F08003755E01AE56AF57AC54AD55AE
:104D5F00EF2DFDEE3CFC74028C068D071200398E90
:104D6F00568F579000AEE060099000AEE0C3943DBF
:104D7F004002804390001BE0FEA3E0FF9000AEE0F6
:104D8F008E048F05FF12693B74018C068D0712008C
:104D9F003990001FEEF0A3EFF090001FE0F8A3E0B2
:104DAF0090001DC8F0A3C8F090001BE4F0A3F0C260
:104DBF001EE5B554FBF5B5A2B4B34002C227A2A4B9
:104DCF00B34002C226A2A3B34002C228A225B34019
:104DDF0002C225A221B34006A22392228002B22250
:104DEF00900096E06012E56D700EA221B35009A2FB
:104DFF0022302301B3B3400280067405900050F0B7
:104E0F00C221803AAE56AF57AC54AD55EF2DFDEEE3
:104E1F003CFC74018C068D071200398E568F57E5B6
:104E2F006DC39402500DAC54AD557488C39D74136B
:104E3F009C400280091241F07406900050F0E55E2C
:104E4F00B423127403900050F0D2259000CBE0B43D
:104E5F0001031241F0AE58AF59AC54AD55EF2DFDD3
:104E6F00EE3CFC8C588D59AE54AF55EFD39DEE9C54
:104E7F004011900013E0FAA3E0FBEBC394E8EA942F
:104E8F000340028006900013126959900010E0FE53
:104E9F00A3E0FFAC54AD55EF2DFDEE3CFC900010A0
:104EAF00ECF0A3EDF09000CBE0B40118AE54AF5589
:104EBF00740512694B740112003990000CEEF0A3C7
:104ECF00EFF08011AE54AF55740212694B90000C85
:104EDF00EEF0A3EFF0C28E758D00758B0075640038
:104EEF00755501755400D28EE55E240875F009845E
:104EFF00AFF07E00EF4E7075900010E0F8A3E090D9
:104F0F00000EC8F0A3C8F090000EE0FEA3E0FFEF84
:104F1F004E600B7C7F7D8A1268398E528F539000C2
:104F2F0010E4F0A3F0AE52AF537428BE00039F50AD
:104F3F0010E5632FFF50010E74011200398E528F4E
:104F4F00538553639000D2E0A852B8000DD3955308
:104F5F004008E55390004FF080099000D2E0149084
:104F6F00004FF0E56D60067553007552009000C953
:104F7F00E0B40308900046E0655E6002800BA22259
:104F8F00B34004D2248002B224E55E640B6005E5D1
:104F9F005EB41D099000BBE060031223D29000C0E5
:104FAF00E0B4011490004DE0655E600790004EE0A4
:104FBF00B55E03756F00801E90004DE0655E601357
:104FCF0090004DE0240C655E600990004DE02418C0
:104FDF00B55E03756F00A213B35006A212B3B340B0
:104FEF0003025098900087E0B40173900109E0B478
:104FFF000214120E2690007AE075F0BEA4FFAEF0F8
:10500F008E5C8F5D8056E56775F00A84FF7E009099
:10501F000581126972E0F55B755A00AE5AAF5B906D
:10502F0000ACE012694B74648E048F05FF12693B6C
:10503F008C5C8D5DE55D900012F0AE5AAF5B900019
:10504F0085E012694B74648E048F05FF12693B74FF
:10505F00BE8C068D0712694B8E5C8F5D801790009A
:10506F0085E075F0BEA4FFAEF08E5C8F5D9000AC56
:10507F00E0900012F0E561C394CC5006E55D455C0D
:10508F00700280031242F6D213E56DB40106E55E9D
:10509F00640B600280097570019000517401F0E596
:1050AF006D600302513E9000CEE0600D900079E0FC
:1050BF00A852B800069553400280409000CEE0B44D
:1050CF00021F900043E0655E600F900044E0655E54
:1050DF006007900045E0B55E03757003756C008046
:1050EF000CC200756C00900019E4F0A3F0900079E9
:1050FF00E060067409900050F08034900043E0B5F2
:10510F005E0B7570019000517401F0802290004485
:10511F00E0B55E0B7570017402900051F080109035
:10512F000045E0B55E097570017403900051F0A25F
:10513F0010B3920EA210B330B601B3500302530155
:10514F00756E019000AEE0B43D13A210B34008E5B8
:10515F00B54404F5B58006E5B554FBF5B5E5B544A2
:10516F0001F5B5741C900071F0A210920EE55ED39C
:10517F00944A4014D212E55ED3946D400B740490A0
:10518F000050F0D225755E469000D6E0B40107E5D9
:10519F006AC39414400280091241F07413900050B6
:1051AF00F0A22D300301B35017A22DB34008E5B57F
:1051BF004408F5B58006E5B554F7F5B5A22D920371
:1051CF00A22E300401B35017A22EB34008E5B54408
:1051DF0002F5B58006E5B554FDF5B5A22E9204A2F1
:1051EF002F300501B3500FA22FB34004D297800286
:1051FF00C297A22F9205A230300601B3500FA230F2
:10520F00B34004D2A28002C2A2A2309206A23130D1
:10521F000701B3500FA231B34004D2A18002C2A143
:10522F00A2319207A232300801B35017A232B34015
:10523F0008E5B54440F5B58006E5B554BFF5B5A210
:10524F00329208A233300901B35017A233B340088A
:10525F00E5B54480F5B58006E5B5547FF5B5A233C5
:10526F009209A234300A01B3500FA234B34004D2D2
:10527F00928002C292A234920AA235300B01B3502F
:10528F000FA235B34004D2878002C287A235920B9A
:10529F00A236300C01B3500FA236B34004D2908027
:1052AF0002C290A236920CE56AC394415009740E63
:1052BF00900050F01241F0900058E0FE900054E042
:1052CF0004C39E4009900054E0D39408400974FB36
:1052DF00900050F01241F090005DE0601590005D7D
:1052EF00E0FE900057E06E600974FE900050F012DF
:1052FF0041F0A225B34006C296C295C2A090010606
:10530F00E0600CAE52AF537414BE00059F40028094
:10531F004890008EE09062CEF8282873803BA2B4AC
:10532F00B35005A227B34002800512433ED2278017
:10533F0028A2A3B35005A228B34002800512433E12
:10534F00D2288015A2A4B35005A226B3400280052F
:09535F0012433ED22680028000B8
:1062CE0002532B02532D02534002535302536602C4
:0262DE00536803
:10536800A215B3B35008900046E0655E600302538F
:10537800FDA201B35006A200B3B3400280719000B1
:10538800C9E0B40343123A67A20DB34021A224B383
:105398004005123AC38003123AE49000E7E0B401F2
:1053A8000BA202B34004D2A18002C2A18018123A13
:1053B800C3123AE49000E7E0B4010BA202B3400440
:1053C800D2A18002C2A180249000E7E0C3940250D9
:1053D8000F123A67123AC3A202B34002D292800C6B
:1053E800123A67123AC3123A97123AE475A700C202
:1053F80015D216D217A216B3B35008900047E0652D
:105408005E6003025492A201B35006A200B3B340F7
:105418000280719000C9E0B40343123A67A20DB349
:105428004021A224B34005123ACE8003123AEF90ED
:1054380000E7E0B4010BA202B34004D2A18002C28B
:10544800A18018123ACE123AEF9000E7E0B4010BAF
:10545800A202B34004D2A18002C2A180249000E736
:10546800E0C39402500F123A67123ACEA202B34038
:1054780002D287800C123A67123ACE123A97123A41
:10548800EF75A700D215C216D217A217B3B35008EA
:10549800900048E0655E6003025527A201B35006FC
:1054A800A200B3B3400280719000C9E0B403431274
:1054B8003A67A20DB34021A224B34005123AD9801D
:1054C80003123AFA9000E7E0B4010BA202B34004D9
:1054D800D2A18002C2A18018123AD9123AFA9000D9
:1054E800E7E0B4010BA202B34004D2A18002C2A13A
:1054F80080249000E7E0C39402500F123A67123AF2
:10550800D9A202B34002D290800C123A67123AD95B
:10551800123A97123AFA75A700D215D216C217E5B1
:0F552800709062E0F8282873025A379000BCE0B8
:0662E000025530025533A7
:10553700906313F8282873121EAE8012121EAE80D5
:0E5547000D121F388008121FE48003121FE4AB
:0F63130002553E02554302554802554D02555260
:10555500757002025A37122110122227A23BB3405E
:10556500229000B0E0F56C900081E0256CFE900083
:105575004FE075F01E84FC7F00EE2CF5367410901C
:105585000050F09007B9E0FEA3E0FF740A12694BE2
:1055950090000EE0FCA3E0FD74098F02FF12693B49
:1055A5008D078C038E048A058B061268399007BD1A
:1055B500EEF0A3EFF074F0BE00039F500B74F09073
:1055C50007BDF8E4F0E8A3F0E53670037536019001
:1055D50007BDE0FEA3E0FFE5362FFF50010E900763
:0D55E500BDEEF0A3EFF0757003900051E0F3
:0362E60002555B03
:1055F200906322F82828738019A23C400375700A30
:105602008010A23C400375700B8007A23C400375DA
:02561200700C1A
:0C6322000255F90255FB02560402560D0C
:10561400025A379006C8E060031224EA900107E0BA
:10562400B40114900108E0A852B80004955350073F
:10563400E55FC39560400280097415900050F00244
:1056440056C79000BCE0D39402403F900090E02401
:1056540003A852B8000495535009900092E0D395E2
:105664006150028008D2017408900050F0900090BC
:10567400E0A852B80005D39553500B900092E02453
:1056840003C395615002C2018039900090E0240365
:10569400A852B8000495535007E55FC395604002D3
:1056A4008008D2017408900050F0900090E0A85255
:1056B400B80005D395535009E560240FC3955F5096
:1056C40002C2019000D6E07007E56AC39414400258
:1056D4008002D201A2014005757004800A75701021
:1056E400900019E4F0A3F0A20DB34029E56775F02A
:1056F4000A84FF7E00900581126972E0C3946950A8
:1057040005122407800F9007BBE0F8A3E09007B9C7
:0C571400C8F0A3C8F0025A379000BCE0B7
:0662E90002561702571CCB
:1057200090632EF8282873120F108012120F108029
:0E5730000D1210BE800812117080031211704D
:0F632E0002572702572C02573102573602573BAE
:10573E009006CCE060031225C6757005025A37122A
:10574E0012B07570069006D0E060031226B6900671
:10575E00D4E06003122792025A37900012E06006DE
:10576E00A20DB3B34002801D900012E02529FFAEBA
:10577E002850010E8E288F29E55ED3941250069084
:10578E000012E014F01214F67570079006D8E0605F
:10579E000312286E9006DCE0600312294A025A3783
:1057AE00900109E0B40203120E9E1218F5757008EE
:1057BE009006E0E06003122A269006E4E0600312F1
:1057CE002B02025A37121CB1A215B35005A216B302
:1057DE0040028006D215D216D2177570109006E8C8
:1057EE00E06003122BDE9006ECE06003122CBA028E
:1057FE005A37025A37900039E0C394465008C29681
:10580E007446900039F0900049E0B4011DE536244D
:10581E000AF5369007BDE0FEA3E0FF740A2FFF5095
:10582E00010E9007BDEEF0A3EFF0900049E0B40238
:10583E001DE5362414F5369007BDE0FEA3E0FF7497
:10584E00142FFF50010E9007BDEEF0A3EFF085363A
:10585E005B755A00900043E0F573123B05E55D90D1
:10586E000039F0900006E55AF0A3E55BF0E5739081
:10587E00003AF0C2199007BDE0F55AA3E0F55B902F
:10588E000043E0F573123B05E55D900037F09000A4
:10589E0000E55AF0A3E55BF0E573900038F0C2180E
:1058AE00E56DB4010575700B8003757003025A37F0
:1058BE0090003DE0C394465008C295744690003D5A
:1058CE00F090004AE0B4011DE536240AF536900743
:1058DE00BDE0FEA3E0FF740A2FFF50010E9007BD3E
:1058EE00EEF0A3EFF090004AE0B4021DE53624146A
:1058FE00F5369007BDE0FEA3E0FF74142FFF5001B4
:10590E000E9007BDEEF0A3EFF085365B755A009052
:10591E000044E0F573123B05E55D90003DF090000C
:10592E0008E55AF0A3E55BF0E57390003EF0C21B6C
:10593E009007BDE0F55AA3E0F55B900044E0F573E7
:10594E00123B05E55D90003BF0900002E55AF0A396
:10595E00E55BF0E57390003CF0C21AE56DB401050D
:10596E0075700C8003757003025A37900041E0C3C6
:10597E0094465008C2A07446900041F090004BE04F
:10598E00B4011DE536240AF5369007BDE0FEA3E00E
:10599E00FF740A2FFF50010E9007BDEEF0A3EFF03B
:1059AE0090004BE0B4021DE5362414F5369007BD89
:1059BE00E0FEA3E0FF74142FFF50010E9007BDEE22
:1059CE00F0A3EFF085365B755A00900045E0F57355
:1059DE00123B05E55D900041F090000AE55AF0A3F8
:1059EE00E55BF0E573900042F0C21D9007BDE0F557
:1059FE005AA3E0F55B900045E0F573123B05E55DBB
:105A0E0090003FF0900004E55AF0A3E55BF0E573DB
:105A1E00900040F0C21CE56DB40103756D00757009
:095A2E0003800680048002800060
:1062EF0002574D0257680257AE0257D302580002A9
:1062FF0058030258BE025979025A31025A33025AD0
:04630F0035025A37C2
:105A3700900037E0B55E028003025AD9A21840727F
:105A4700900000E0FEA3E0FFEF4E6021AE56AF5797
:105A5700900000E0FCA3E0FD120003740A8E048F9F
:105A670005FF12693B900000ECF0A3EDF0900038C1
:105A7700E0601A900000E0FEA3E0FFAC56AD57EFE0
:105A87002DFDEE3CFC900000ECF0A3EDF09000380B
:105A9700E0D39401401A900000E0FEA3E0FFAC566B
:105AA700AD57EF2DFDEE3CFC900000ECF0A3EDF0C0
:105AB700D218AE54AF55900000E0FCA3E0FDEFC351
:105AC7009DEE9C400D124385D296C21874C8900073
:105AD70037F0A218B3B35007900037E0B55E0280E5
:105AE7000D124385D29674C8900037F0C218900003
:105AF70039E0B55E028003025B94A2194072900000
:105B070006E0FEA3E0FFEF4E6021AE56AF579000D0
:105B170006E0FCA3E0FD120003740A8E048F05FF64
:105B270012693B900006ECF0A3EDF090003AE060BC
:105B37001A900006E0FEA3E0FFAC56AD57EF2DFD2F
:105B4700EE3CFC900006ECF0A3EDF090003AE0D3B9
:105B57009401401A900006E0FEA3E0FFAC56AD5753
:105B6700EF2DFDEE3CFC900006ECF0A3EDF0D21912
:105B7700AE54AF55900006E0FCA3E0FDEFC39DEEE9
:105B87009C400AC2967446900039F0C219A219B314
:105B9700B35007900039E0B55E02800AC29674469A
:105BA700900039F0C21990003BE0B55E0280030215
:105BB7005C4FA21A4072900002E0FEA3E0FFEF4E96
:105BC7006021AE56AF57900002E0FCA3E0FD120043
:105BD70003740A8E048F05FF12693B900002ECF0F4
:105BE700A3EDF090003CE0601A900002E0FEA3E015
:105BF700FFAC56AD57EF2DFDEE3CFC900002ECF0EC
:105C0700A3EDF090003CE0D39401401A900002E02D
:105C1700FEA3E0FFAC56AD57EF2DFDEE3CFC900028
:105C270002ECF0A3EDF0D21AAE54AF55900002E0AB
:105C3700FCA3E0FDEFC39DEE9C400D124385D2957A
:105C4700C21A74C890003BF0A21AB3B35007900071
:105C57003BE0B55E02800D124385D29574C8900073
:105C67003BF0C21A90003DE0B55E028003025D0A78
:105C7700A21B4072900008E0FEA3E0FFEF4E6021F8
:105C8700AE56AF57900008E0FCA3E0FD1200037486
:105C97000A8E048F05FF12693B900008ECF0A3ED14
:105CA700F090003EE0601A900008E0FEA3E0FFAC31
:105CB70056AD57EF2DFDEE3CFC900008ECF0A3ED40
:105CC700F090003EE0D39401401A900008E0FEA354
:105CD700E0FFAC56AD57EF2DFDEE3CFC900008EC15
:105CE700F0A3EDF0D21BAE54AF55900008E0FCA333
:105CF700E0FDEFC39DEE9C400AC295744690003DBF
:105D0700F0C21BA21BB3B3500790003DE0B55E0283
:105D1700800AC295744690003DF0C21B90003FE098
:105D2700B55E028003025DC5A21C4072900004E0CC
:105D3700FEA3E0FFEF4E6021AE56AF57900004E0A0
:105D4700FCA3E0FD120003740A8E048F05FF12699D
:105D57003B900004ECF0A3EDF0900040E0601A9057
:105D67000004E0FEA3E0FFAC56AD57EF2DFDEE3C7F
:105D7700FC900004ECF0A3EDF0900040E0D3940118
:105D8700401A900004E0FEA3E0FFAC56AD57EF2D9C
:105D9700FDEE3CFC900004ECF0A3EDF0D21CAE54F9
:105DA700AF55900004E0FCA3E0FDEFC39DEE9C40DF
:105DB7000D124385D2A0C21C74C890003FF0A21CEC
:105DC700B3B3500790003FE0B55E02800D124385E4
:105DD700D2A074C890003FF0C21C900041E0B55EAD
:105DE700028003025E80A21D407290000AE0FEA3BB
:105DF700E0FFEF4E6021AE56AF5790000AE0FCA3DC
:105E0700E0FD120003740A8E048F05FF12693B90B0
:105E1700000AECF0A3EDF0900042E0601A90000A4F
:105E2700E0FEA3E0FFAC56AD57EF2DFDEE3CFC9036
:105E3700000AECF0A3EDF0900042E0D39401401A81
:105E470090000AE0FEA3E0FFAC56AD57EF2DFDEE44
:105E57003CFC90000AECF0A3EDF0D21DAE54AF5518
:105E670090000AE0FCA3E0FDEFC39DEE9C400AC250
:105E7700A07446900041F0C21DA21DB3B350079015
:105E87000041E0B55E02800AC2A07446900041F06E
:105E9700C21D9000D9E0B402028003025FB59000F2
:105EA70073E0D395665064900073E0F4042566FEB2
:105EB7009000DCE08E00F5F0E884FF7E008F73EF42
:105EC700C39410500CEF8573F0A4FDACF08D738074
:105ED700037573FF900073E0D39573400B900073C5
:105EE700E0C39573F57180037571009000F7E0D3F7
:105EF700957140069000F7E0F5719000F8E0C395C2
:105F07007150069000F8E0F5718071900073E0C35E
:105F17009566FE9000DCE08E00F5F0E884FF7E00D9
:105F27008F73EFC39410500CEF8573F0A4FDACF0A2
:105F37008D7380037573FF85735B755A00900073CB
:105F4700E0255BFFAE5A50010E8E5A8F5B74FFBE81
:105F57000009D39F4005855B7180037571FF900031
:105F6700F7E0D3957140069000F7E0F5719000F8DF
:105F7700E0C3957150069000F8E0F571A20DB3B338
:105F8700500D900074E0FE9000E4E0D39E50028034
:105F97000A7407900050F0C2A2801375A710E5CDD0
:105FA700C395714004C2A28002D2A275A7009000D7
:105FB700FEE0A852B80005D3955350169000FDE0B7
:105FC700A852B8000D955340099000FFE0D39561A2
:105FD7004002802575A710A20DB3B35007E5CDC3C6
:105FE70094BF40028008E5B54410F5B58006E5B5D5
:105FF70054EFF5B575A700802375A710A20DB3B3AD
:106007005007E5CDC3944040028008E5B54410F53C
:10601700B58006E5B554EFF5B575A700E56FC394F0
:1060270009500AA2EDB34005C2ED123050AE54AF8D
:10603700557498C39F743A9E400C900072E0C394C5
:106047005A40030262A7A212B340091241F0740634
:10605700900050F0A220B34008E5B54404F5B580A0
:1060670006E5B554FBF5B5A214B3500EE561D3941C
:10607700334007E561C394CC40028041900109E0B9
:10608700B40214120E2690007AE075F050A4FFAE09
:10609700F08E5C8F5D800F900085E075F050A4FF57
:1060A700AEF08E5C8F5DE55D455C6011E5B5440142
:1060B700F5B5741C900071F01242F6D2149000727C
:1060C700E0D394014007E561C3941A40028002C2FD
:1060D700149006C8E060031224EAA22D300301B32E
:1060E7005017A22DB34008E5B54408F5B58006E57D
:1060F700B554F7F5B5A22D92039006CCE0600312D4
:1061070025C6A22E300401B35017A22EB34008E5CE
:10611700B54402F5B58006E5B554FDF5B5A22E9256
:10612700049006D0E060031226B6A22F300501B313
:10613700500FA22FB34004D2978002C297A22F928A
:10614700059006D4E06003122792A230300601B30F
:10615700500FA230B34004D2A28002C2A2A2309252
:10616700069006D8E0600312286EA231300701B30B
:10617700500FA231B34004D2A18002C2A1A2319232
:10618700079006DCE0600312294AA232300801B307
:106197005017A232B34008E5B54440F5B58006E58F
:1061A700B554BFF5B5A23292089006E0E06003123D
:1061B7002A26A233300901B35017A233B34008E5AA
:1061C700B54480F5B58006E5B5547FF5B5A23392A1
:1061D700099006E4E06003122B02A234300A01B3EF
:1061E700500FA234B34004D2928002C292A23492DA
:1061F7000A9006E8E06003122BDEA235300B01B3EC
:10620700500FA235B34004D2878002C287A23592CD
:106217000B9006ECE06003122CBAA236300C01B3E7
:10622700500FA236B34004D2908002C290A2369299
:106237000C900072E0C3945A5010E56FB4090990AE
:106247000072E004F0756F00803BE56FB4090375D9
:106257006F00755500755400758D00758B0075645A
:1062670000900071E0C3942A5008900071E004F098
:106277008006742A900071F0900071E0B42A06E558
:10628700B554FEF5B5900072E0D394014007E56A76
:10629700C3944140028009740E900050F01241F0FF
:0362A700024AB2F6
:10633D000000010001400160018001A001C001E0E9
:10634D0002000300039603B603D603F40400050010
:10635D000512052405360548055A056C057E059080
:10636D0005A805C005DE0600061406280646066EBD
:10637D0006AE05CF00FF013F015F017F019F01BF09
:10638D0001DF01FF02FF039503B503D503F303FFFF
:10639D0004FF05110523053505470559056B057DD9
:1063AD00058F05A705BF05CE05F106130627064582
:1063BD00066D06AD06ED05DD0FAA0FA50F9F0F9A11
:1063CD000F940F8D0F870F800F780F710F680F606F
:1063DD000F570F4E0F450F3B0F300F250F1A0F0E96
:1063ED000F020EF50EE80EDB0ECC0EBE0EAE0E9F9E
:1063FD000E8E0E7D0E6C0E5A0E470E340E200E0CA8
:10640D000DF70DE20DCB0DB50D9D0D850D6D0D54DB
:10641D000D3A0D200D050CE90CCE0CB10C940C763B
:10642D000C580C3A0C1B0BFB0BDB0BBB0B9A0B79B3
:10643D000B570B350B130AF10ACE0AAB0A870A6408
:10644D000A400A1C09F809D409B0098C09670943E7
:10645D00091F08FB08D608B2088E086A08460823EB
:10646D0007FF07DC07B9079607730751072F070DBD
:10647D0006EC06CA06AA068906690649062A060A10
:10648D0005EC05CD05B0059205750558053C0520B3
:10649D00050504EA04CF04B5049C04820469045183
:1064AD0004390422040B03F403DE03C803B2039D75
:1064BD00038903750361034D033B0328031603048E
:1064CD0002F202E102D102C002B002A002910282E8
:1064DD000273026502570249023C022F0222021684
:1064ED00020901FD01F201E601DB01D001C601BB8C
:1064FD0001B101A7019D0194018B01820179017008
:10650D000168016001580150014801410139013212
:10651D00012B0125011E01180111010B010500FFC1
:10652D0000FA0FA60FA00F990F920F8B0F840F7CFF
:10653D000F740F6B0F620F580F4E0F430F380F2C48
:10654D000F1F0F120F050EF70EE80ED80EC80EB75F
:10655D000EA50E930E800E6C0E580E420E2C0E15BF
:10656D000DFD0DE40DCB0DB10D950D790D5D0D3FAF
:10657D000D200D010CE10CC00C9E0C7C0C590C3542
:10658D000C100BEA0BC40B9E0B760B4F0B260AFD62
:10659D000AD40AAA0A800A550A2A09FF09D409A8A9
:1065AD00097C0950092508F908CD08A10875084A84
:1065BD00081E07F307C8079D07730749072006F74D
:1065CD0006CE06A6067E06570630060A05E405BF6A
:1065DD00059B057705540532051004EF04CE04AE76
:1065ED00048F047104530435041903FD03E203C73A
:1065FD0003AD0394037B0363034B0334031E0308B2
:10660D0002F302DE02CA02B602A30291027F026DFC
:10661D00025C024C023C022C021D020E020001F231
:10662D0001E401D701CA01BE01B101A6019A018F92
:10663D000185017A01700166015D0153014A014135
:10664D00013901310129012101190112010B010447
:10665D0000FD00F700F000EA00E400DE00D900D3F1
:10666D0000CE00C900C400BF00BA00B500B100AD36
:10667D0000A800A400A0009C009900950091008E38
:0C668D00008A008700840081007E007BF2
:10009E007547009007C5E4F0A3F075310075300088
:1000AE00754D00754E00C238D23974FE9007C7F8F0
:1000BE00E4F0E8A3F074FE9007C9F8E4F0E8A3F0CA
:1000CE0074FE9007D3F0745A9007D4F0745A9007C8
:1000DE00D5F0D23AC22CC23CC23722750B00750A3B
:1000EE0000AE0AAF0BAC08AD09EDC39FEC9E4016F7
:1000FE0074FF12692B75CF01780B740126F650042C
:10010E0018E436F650DB2290004CE0B4AA1C90079F
:10011E0081E0B43C159007C1E0FEA3E0FFEF4E6016
:10012E0009741EBE0004D39F5003020243755D0086
:10013E00755C0075F8099007C1E0FEA3E0FF740737
:10014E006F4E6006740E6F4E7006743A900781F013
:10015E009007C1E0FEA3E0FF7408BE001ED39F40CF
:10016E001A7E017F089007C1E0FCA3E0FD1DBDFFD4
:10017E00011C1200038E5A8F5B801F9007C1E0FE98
:10018E00A3E0FF740812698F8F048E057E017F082D
:10019E00CDCCCD1200038E5A8F5BAE5CAF5D740C6E
:1001AE00D39F74019E500302023EA2F9B3407EE536
:1001BE005D455C700375A382AE5CAF5D74016F4EDE
:1001CE00700375A300AE5CAF5D74026F4E700D9040
:1001DE0007C2E075F002A4FDACF08DA3AE5CAF5D7E
:1001EE0074036F4E700375A300AE5CAF5D7403BEF7
:1001FE0000039F5013AC5AAD5BED2FFFEC3EFE900B
:10020E00007D126972E0F5A3AE5CAF5DEFB40B0931
:10021E00EEB40105741412692BAE5CAF5DEFB40B36
:10022E0007EEB4010375F80D785C12699F0201A800
:10023E0090004CE4F022755D00755C0075F8099035
:10024E0007C1E0FEA3E0FF7408BE001ED39F401A54
:10025E007E017F089007C1E0FCA3E0FD1DBDFF01FC
:10026E001C1200038E5A8F5B801F9007C1E0FEA305
:10027E00E0FF740812698F8F048E057E017F08CD12
:10028E00CCCD1200038E5A8F5BAE5CAF5D7411D372
:10029E009F74019E5003020374A2F9B3500302032C
:1002AE0071E55D455C700375A3D2AE5CAF5D740104
:1002BE006F4E700375A300AE5CAF5D74026F4E702F
:1002CE000D9007C2E075F002A4FDACF08DA3AE5CFC
:1002DE00AF5D74036F4E700375A300AE5CAF5D74BB
:1002EE00046F4E700375A300AE5CAF5D74056F4E68
:1002FE00700375A300AE5CAF5D74066F4E70037530
:10030E00A300AE5CAF5D74076F4E700375A300AEB5
:10031E005CAF5D74086F4E700375A300AE5CAF5D8D
:10032E007408BE00039F5016AC5AAD5BED2FFFEC68
:10033E003EFE900078126972E5A3F075A300AE5CE4
:10034E00AF5DEFB41009EEB40105741412692BAE53
:10035E005CAF5DEFB41007EEB4010375F80D785C79
:10036E0012699F02029722755D00755C0075F8098F
:10037E00AE5CAF5D7417BE0004D39F500302044DF4
:10038E00A2F9B3500302044AE55D455C700375A300
:10039E00D2AE5CAF5D74016F4E700375A300AE5CA0
:1003AE00AF5D74026F4E700D9007C2E075F002A43F
:1003BE00FDACF08DA3AE5CAF5D74036F4E70037534
:1003CE00A300AE5CAF5D74046F4E700375A300AEF8
:1003DE005CAF5D74056F4E700375A300AE5CAF5DD0
:1003EE0074066F4E700375A300AE5CAF5D74076F3D
:1003FE004E700375A300AE5CAF5D74086F4E700354
:10040E0075A300AE5CAF5D7408BE00039F500C90E8
:10041E00005A126972E5A3F075A300AE5CAF5D746D
:10042E00166F4E7005741412692BAE5CAF5D7416A8
:10043E006F4E700375F80D785C12699F02037E2271
:10044E0090004CE0B4AB0280030204E8755D0075C9
:10045E005C0075F809AE5CAF5D7412BE007CD39F74
:10046E004078A2F9B34070E55D455C700375A382D8
:10047E00AE5CAF5D74016F4E700375A300AE5CAFE2
:10048E005D74026F4E700D9007C2E075F002A4FD10
:10049E00ACF08DA3AE5CAF5D74036F4E700375A3AD
:1004AE0000AE5CAF5D7403BE00039F500990005F09
:1004BE00126972E0F5A3AE5CAF5D74116F4E7005FC
:1004CE00741412692BAE5CAF5D74116F4E700375B0
:1004DE00F80D785C12699F020463229007D0E4F055
:1004EE0074649007C1F8E4F0E8A3F012037574C8C1
:1004FE009007C1F8E4F0E8A3F074FF90005AF0748E
:10050E00FF90005BF074FF90005CF074009000545C
:10051E00F074FF90005DF0740090005FF074019035
:10052E000060F0900066E0B4371A900063E090002F
:10053E005AF0900064E090005BF0900065E090004F
:10054E005CF080469007D07401F074659007C1F896
:10055E00E4F0E8A3F012037574C89007C1F8E4F054
:10056E00E8A3F0900066E0B4371A900063E09000C4
:10057E005AF0900064E090005BF0900065E090000F
:10058E005CF0800674029007D0F09007D1E4F0740E
:10059E00669007C1F8E4F0E8A3F012037574C890F2
:1005AE0007C1F8E4F0E8A3F0900065E0B4371290CC
:1005BE000063E0900054F0900064E090005DF080E5
:1005CE00769007D17401F074679007C1F8E4F0E8F3
:1005DE00A3F012037574C89007C1F8E4F0E8A3F015
:1005EE00900065E0B43712900063E0900054F090F4
:1005FE000064E090005DF0803E74029007D1F074CC
:10060E00689007C1F8E4F0E8A3F012037574C8907F
:10061E0007C1F8E4F0E8A3F0900065E0B43712905B
:10062E000063E0900054F0900064E090005DF08074
:10063E000674039007D1F022E54E64046006E59936
:10064E0064FF60028031A2384004D2388027E54E24
:10065E00600874E6254E900050F0E54D600874F089
:10066E00254D900050F0E54EB4010280FE754E000F
:10067E00754D00C2388002C238E54E90384AF828CF
:10068E002873754E00E599B4FF03754D01E599B4D5
:10069E00FE03754D02E599B4FD03754D03E599B45E
:1006AE00FC03754D04E599B4FA03754D05E599B44F
:1006BE00FB06754E011241F0E599B4F906754E042C
:1006CE001241F0E599D394E54007E599C394F040C3
:1006DE0002801685994F754E027E017F00E54FC34D
:1006EE0094E612694B8E328F339007C5E4F0A3F077
:1006FE00E599D394C44007E599C394E64002802857
:10070E0085994F754E0374E5C3954FF533753200D9
:10071E00AE32AF3390633D12691AE493F8740193CD
:10072E009007C5C8F0A3C8F0D299020C569000638A
:10073E00E07005A22AB3400280429007C5E0FEA3F6
:10074E00E0FF74FFBE00039F5009EFC39446EE9482
:10075E000640119007C5E0FEA3E0FFEFD3946DEEC7
:10076E00940640139007C5E0FEA3E0FF90008112AF
:10077E006972E599F0800385997480119007C5E040
:10078E00FEA3E0FF900081126972E599F09007C513
:10079E001269599007C5E0FEA3E0FFEFB40106EE23
:1007AE00B4070280030209FD900781E0B43C028089
:1007BE00030209FDA22A50030208E8C29C900063BE
:1007CE00E090011FF0900064E090008EF0900065C4
:1007DE00E09000AEF0900066E09000D7F0900067D9
:1007EE00E0900083F0900068E09000C9F0900069FE
:1007FE00E09000E7F090006AE09000BBF090006B94
:10080E00E09000D9F090006CE0900109F090006D3E
:10081E00E090016DF090006EE090016EF090006F30
:10082E00E090016FF0123B9C900075E09000F0F0AC
:10083E00900076E09000A7F0900077E09000A8F08E
:10084E0074639007C1F8E4F0E8A3F074AB90004C29
:10085E00F012044E90004CE4F07464F50975080033
:10086E001200E9A21F4039757301E573D394075046
:10087E002DE5739007C1F8E4F0E8A3F074AA900098
:10088E004CF0120115E573C39407500A7464F50910
:10089E007508001200E97873740126F650CC803783
:1008AE00757308E573D3940E502DE5739007C1F858
:1008BE00E4F0E8A3F074AA90004CF0120115E57371
:1008CE00C3940E500A7464F5097508001200E97895
:1008DE0073740126F650CC0209E7C29C90011FE00A
:1008EE00900063F090008EE0900064F09000AEE017
:1008FE00900065F09000D7E0900066F0900083E0E5
:10090E00900067F09000C9E0900068F09000E7E07A
:10091E00900069F09000BBE090006AF09000D9E082
:10092E0090006BF0900109E090006CF07400900064
:10093E006DF0740090006EF0740090006FF07463B0
:10094E009007C1F8E4F0E8A3F074AB90004CF012FD
:10095E00044E90004CE4F07464F509750800120022
:10096E00E9757301E573D394075026E5739007C1BB
:10097E00F8E4F0E8A3F074AA90004CF0120115749C
:10098E0064F5097508001200E97873740126F650B3
:10099E00D3D29C7599FB743C900781F0757308E572
:1009AE0073D3940E5026E5739007C1F8E4F0E8A3D4
:1009BE00F074AA90004CF01201157464F5097508D4
:1009CE00001200E97873740126F650D374C89007AC
:1009DE00C1F8E4F0E8A3F080FE74C89007C1F8E413
:1009EE00F0E8A3F0D29C754E00754D007599FB0290
:1009FE000C569007C5E0FEA3E0FFEF4E70068599FA
:100A0E00317530009007C5E0FEA3E0FF74016F4E14
:100A1E00701BAC30AD31AA32AB33ED2BFBEC3AFA96
:100A2E008A068B07900081126972E599F09007C5CE
:100A3E001269599007C5E0FEA3E0FF74026F4E7075
:100A4E0021AC30AD3174566D4C7006E54F64E660E6
:100A5E000280031241F0123B9C854F99754E007532
:100A6E004D00020C569007C5E0FEA3E0FF900081FA
:100A7E00126972E599F09007C51269599007C5E0A1
:100A8E00FEA3E0FFAC32AD338F028E038C068D07D2
:100A9E0090638112691AE493F9740193FEEAD39E6E
:100AAE00EB994009854F99754E00754D00020C5615
:100ABE009007C5E0FEA3E0FF900081126972E599F0
:100ACE00F09007C51269599007C5E0FEA3E0FFEF4D
:100ADE00B40006EEB401028003020C5690005CE0F6
:100AEE00D394C7400B90005CE0C394C8F550801AB5
:100AFE0090005CE0D39463400B90005CE0C3946480
:100B0E00F550800690005CE0F550E55075F002A4BB
:100B1E00FFAEF08F73EF90008112697DEFFCE0FD68
:100B2E00EC90008412697DEDFCE0FDEC2DB55002D9
:100B3E008003020C470FEF90008112697DE573FF71
:100B4E00E0FCEF90008512697DECFFE0FCEFC39CAA
:100B5E00B550028003020C47E57390008312697D45
:100B6E00E573FFE0FCEF90008612697DECFFE0FC80
:100B7E00EF2CB550028003020C47E57390008712EC
:100B8E00697DE0C39550900063F0E5739000881284
:100B9E00697DE0C39550900064F0E5739000891272
:100BAE00697DE0C39550900065F07400900066F08A
:100BBE0074FF900067F0E57390008B12697DE0C3BF
:100BCE009550900068F0E57390008C12697DE0C33B
:100BDE009550900069F0E57390008D12697DE0C329
:100BEE00955090006AF0E57390008A12697DE0C31B
:100BFE0095509007C1F8E4F0E8A3F074AB90004C68
:100C0E00F012044E7464F5097508001200E990079D
:100C1E00C112695912044E7464F509750800120068
:100C2E00E99007C112695912044E7599F97464F569
:100C3E00097508001200E980FE7599FF7464F509C4
:080C4E007508001200E980FEA8
:0F384A0002069002073B020A00020A73020ABE3E
:100C560022E54D903859F8282873020D699007C58A
:100C6600E0FEA3E0FF900052126972E0F59990074A
:100C7600C51269599007C5E0FEA3E0FF74116F4ED7
:100C86007003754D00020D69856E99020D69900716
:100C9600C5E0FEA3E0FF900081126972E0F599EFCE
:100CA600B40107EEB40703754D009007C5126959E4
:070CB600020D699007C6E082
:0F385900020C60020C63020C8E020C94020CB97C
:100CBD00903A0CF8282873855399020D5E855F993B
:100CCD00020D5E856199020D5E856599020D5E8549
:100CDD006799807D85689980788569998073856A23
:100CED0099806E90001AE0F5998066A239B340079D
:100CFD007599FAC2398041A229B3400575990F80C3
:100D0D00359007D0E0600A9007D0E024DCF599809B
:100D1D00169007D1E0600A9007D1E024DEF59980A6
:100D2D0006900050E0F599900050E4F09007D0E463
:100D3D00F09007D1E4F0C2298017856B9980128558
:100D4D006699800D856C9980087599FC8003754DA9
:010D5D000095
:103A0C00020CC4020CCA020CD0020CD6020CDC0252
:103A1C000CE1020CE6020CEB020CF0020CF8020DAD
:0D3A2C0047020D4C020D51020D56020D5BBC
:0B0D5E009007C51269598003123A3952
:03386800020D66E8
:100D690022E537255BFFAE5A50010E9000811269CA
:100D790072E0F538E537255BFFAE5A50010E0FBF1B
:100D890000010E900081126972E0F539853F3BE55B
:100D990038B539058538378041E539D39538401D4F
:100DA900E539C39538853AF0A4FFAEF0E53B8E04EA
:100DB9008F05FF12693BED2538F537801DE538C3EE
:100DC9009539853AF0A4FFAEF0E53B8E048F05FF17
:100DD90012693BEDF4042538F53722E539D3953806
:100DE900401DE539C39538853AF0A4FFAEF0E53BDF
:100DF9008E048F05FF12693BED2538F537801DE517
:100E090038C39539853AF0A4FFAEF0E53B8E048FDF
:100E190005FF12693BEDF4042538F5372290008768
:100E2900E0B40170E56775F00A84FF7E008F37E54D
:100E39006775F00A84ADF07C008D3A753F0A755AE2
:100E490005755B24E537C394115005120D6A8006B8
:100E59009005B6E0F537E53790007AF0E56775F06B
:100E69000A84FF7E008F37E56775F00A84ADF07C50
:100E7900008D3A753F0A755A05755B5AE537C39473
:100E8900115005120D6A80069005ECE0F537E5373B
:100E9900900012F022900087E0B4016AE56775F0CE
:100EA9000A84FF7E008F37E56775F00A84ADF07C10
:100EB900008D3A753F0A755A05755B36E537C39457
:100EC900115005120D6A80069005C8E0F53785377F
:100ED9004BE56775F00A84FF7E008F37E56775F08B
:100EE9000A84ADF07C008D3A753F0A755A05755B29
:100EF90048E537C394115005120D6A80069005DA4A
:100F0900E0F53785374C22E55F75F00484FF7E00F4
:100F19008F37E55F75F00484ADF07C008D3A753F3D
:100F290004755A01755B00E537C3943F5005120DEE
:100F39006A80069001C0E0F5378537297528009049
:100F4900004FE075F020A4FFAEF09000D2E08E04CF
:100F59008F05FF12693B8D379000BAE0D3955F503A
:100F6900030210169000DEE0D3955F4010ED90016A
:100F7900C112697DE0F52B752A000210139000A9B2
:100F8900E0D3955F4043E5379001C112697DE0F5F3
:100F990038E5379001E112697DE0F5399000DEE02E
:100FA900F404255FF53A9000A9E0FE9000DEE0F434
:100FB900042EF53BE538B539058538378003120D20
:100FC900E485372B752A008041E5379001E11269E4
:100FD9007DE0F538E53790020112697DE0F5399039
:100FE90000A9E0F404255FF53A9000BAE0FE90000C
:100FF900A9E0F4042EF53BE538B539058538378085
:1010090003120DE485372B752A000210BD9000E10B
:10101900E0D3955F5011E53790024112697DE0F503
:101029002B752A000210BD9000AAE0D3955F5043AA
:10103900E53790022112697DE0F538E537900241E4
:1010490012697DE0F5399000AAE0F404255FF53ACC
:101059009000E1E0FE9000AAE0F4042EF53BE538AB
:10106900B539058538378003120DE485372B752A84
:10107900008041E53790020112697DE0F538E537D6
:1010890090022112697DE0F5399000BAE0F4042557
:101099005FF53A9000AAE0FE9000BAE0F4042EF55C
:1010A9003BE538B539058538378003120DE48537B6
:1010B9002B752A00229000F2E0F53C753F11755A14
:1010C90002755B00AE52AF53E53C75F00FA4FDAC61
:1010D900F0EDD39FEC9E4021E53C8E048F05FF1275
:1010E900693BED75F010A4FFAEF0E55F75F0118472
:1010F900FD7C00ED2FF53D800EE55F75F01184FF55
:101109007E00EF24F0F53D853D37E55F75F01184EC
:10111900AFF07E008F3A120D6A85373EAE52AF535B
:101129009000F2E075F00FA4FDACF0EDD39FEC9EBA
:101139004028755A02755B10853D37120D6A853E48
:1011490038853739AE52AF53E53C8E048F05FF120F
:1011590069668D3A853C3B120DE48537297528006F
:10116900752B64752A00229000F2E0F53C753F1159
:10117900755A02755B00AE52AF53E53C75F00FA48A
:10118900FDACF0EDD39FEC9E4021E53C8E048F052C
:10119900FF12693BED75F010A4FFAEF0E56175F043
:1011A9001184FD7C00ED2FF53D800EE56175F01190
:1011B90084FF7E00EF24F0F53D853D37E56175F04C
:1011C9001184AFF07E008F3A120D6A85373EAE5218
:1011D900AF539000F2E075F00FA4FDACF0EDD39F92
:1011E900EC9E4028755A02755B10853D37120D6AD1
:1011F900853E38853739AE52AF53E53C8E048F05AD
:10120900FF1269668D3A853C3B120DE485372975D5
:101219002800E56B6017E56BC394FE50109000E65B
:10122900E0B402099000D4E0D3940B50028017AEC9
:1012390028AF29E56B12694B74E78E048F05FF12FD
:10124900693B8C288D299000BCE0B40453E55F7597
:10125900F00484FF7E008F37E55F75F00484ADF0FC
:101269007C008D3A753F04755A01755B00E537C3FB
:10127900943F5005120D6A80069001C0E0F537AE23
:1012890028AF29E53712694B74648E048F05FF1264
:10129900693BAE28AF29EF2DFDEE3CFC8C288D294A
:1012A900752B64752A0022900087E0B40146E56732
:1012B90075F00A84FF7E008F37E56775F00A84AD03
:1012C900F07C008D3A753F0A755A05755B00E53764
:1012D900C394115005120D6A8006900592E0F53706
:1012E900AE2AAF2BE5372FFF50010E746412698FB8
:1012F9008E2A8F2B900088E0B40146E56875F00AC4
:1013090084FF7E008F37E56875F00A84ADF07C00B4
:101319008D3A753F0A755A05755B6CE537C39411AB
:101329005005120D6A80069005FEE0F537AE2AAF2A
:101339002BE5372FFF50010E746412698F8E2A8FA7
:101349002B900097E0B40249E56AC3944175F00512
:1013590084FF7E008F37E56A75F00584ADF07C0067
:101369008D3A753F05755A06755B00E537C39413C9
:101379005005120D6A8006900694E0F537AE2AAF43
:101389002BE5372FFF50010E746412698F8E2A8F57
:101399002B9000D9E0B40202800302144FE55F7577
:1013A900F01584FF7E008F37E55F75F01584ADF089
:1013B9007C008D3A753F15755A03755BF4E537C3A3
:1013C900940B5005120D6A8006900480E0F537E50C
:1013D9003775F0FFA4FFAEF09000DAE08E048F05B8
:1013E900FF12693BED900073F0E56675F078A4FF94
:1013F900AEF074FF8E048F05FF12693B8C5A8D5B2A
:1014090074028C068D071200398F37AC5AAD5B74A4
:1014190004FF1269668D3A753F04755A06755B2893
:10142900E537C3941D5005120D6A80069006C6E083
:10143900F537AE2AAF2BE5372FFF50010E74641232
:10144900698F8E2A8F2B900086E0B4025DE5617565
:10145900F064A4FFAEF074081200398E5C8F5D74DD
:10146900058E048F05FF12693B8D37AE5CAF5D7445
:10147900058E048F05FF1269668D3A753F05755A09
:1014890005755BDEE537C394135005120D6A8006B6
:10149900900672E0F537AE2AAF2BE5372FFF5001E2
:1014A9000E746412698F8E2A8F2B9000C8E0703CED
:1014B90090004FE075F00584FF7E008F3790004F54
:1014C900E075F00584ADF07C008D3A753F05755ADD
:1014D90005755BC0E537C3941D5005120D6A80067A
:1014E90090065EE0F537E53790007BF02290008F9B
:1014F900E0B401179007CCE0252BFFAE2A50010E6E
:101509009000E3E012698F8E2A8F2B900107E0B4D7
:101519000114900108E0A852B8000495535007E55A
:101529005FC39560400280129000B1E0252BFFAEA9
:101539002A50010E8E2A8F2B802F90008FE0B40342
:1015490016A22CB3B350109007CFE0C39405A8524C
:10155900B800069553400280109000B1E0252BFF9A
:10156900AE2A50010E8E2A8F2B900089E0B4020218
:1015790080030218F490008CE0602FE567D394464D
:101589004028900013E0FEA3E0FF9000C7E075F04B
:1015990003A4FDACF0EFD39DEE9C400E9000EBE070
:1015A900A852B80005D3955350030218F49000BC13
:1015B900E0B40302800302175885615B755A0090F5
:1015C9000093E0A852B800049553500E900094E09F
:1015D900A85AB80005D3955B5003021755E5617504
:1015E900F002A4FFAEF074158E048F05FF12693B5B
:1015F9008C068D07900611126972FEE0FFEE9000CD
:101609008BE0FEEF8E0088F0A4FFAEF074648E04C8
:101619008F05FF12693B8C5A8D5B90004FE075F086
:1016290018A4FFAEF09000D2E08E048F05FF126976
:101639003B8C068D07900629126972AE5AAF5BE0A2
:1016490012694B74648E048F05FF12693B8C5A8DA5
:101659005BE565A85AB80077D3955B4072E565C329
:10166900955BFFE4955AFE8E5A8F5B7428BE000382
:101679009F500C755B28755A00740D900050F0AEA0
:101689005AAF5B90008CE012694B74288E048F0569
:10169900FF12693B8C5A8D5BAE28AF29740A8E0400
:1016A9008F05FF12693B8D068C07AC5AAD5BCFCE17
:1016B900CF120003740A8E048F05FF12693B8C5AFE
:1016C9008D5BAE28AF291269978E288F29807DE519
:1016D90065A85AB80004955B5072AE5AAF5BE565D0
:1016E90012698F8E5A8F5B7428BE00039F500C7548
:1016F9005B28755A00740D900050F0AE5AAF5B909C
:10170900008CE012694B74288E048F05FF12693B27
:101719008C5A8D5BAE28AF29740A8E048F05FF128F
:10172900693B8D068C07AC5AAD5BCFCECF12000357
:10173900740A8E048F05FF12693B8C5A8D5BAE28A3
:10174900AF29EF2DFDEE3CFC8C288D290218F49071
:1017590000D4E0855FF0A4FFAEF0740512694B7404
:10176900071200398E5A8F5B900093E0A852B80097
:101779000495535012900094E075F002A4FDACF06A
:10178900EFC39DEE9C40030218F4E55F75F00B84EE
:10179900FF7E00900611126972FEE0FFEE90008B49
:1017A900E0FEEF8E0088F0A4FFAEF074648E048F23
:1017B90005FF12693B8C5A8D5B90004FE075F0185C
:1017C900A4FFAEF09000D2E08E048F05FF12693BB2
:1017D9008C068D07900629126972AE5AAF5BE0122A
:1017E900694B74648E048F05FF12693B8C5A8D5BBB
:1017F900E565A85AB80077D3955B4072E565C3954E
:101809005BFFE4955AFE8E5A8F5B7428BE00039FD6
:10181900500C755B28755A00740D900050F0AE5A43
:10182900AF5B90008CE012694B74288E048F05FF22
:1018390012693B8C5A8D5BAE28AF29740A8E048FCE
:1018490005FF12693B8D068C07AC5AAD5BCFCECF35
:10185900120003740A8E048F05FF12693B8C5A8D9E
:101869005BAE28AF291269978E288F29807DE5659F
:10187900A85AB80004955B5072AE5AAF5BE5651281
:10188900698F8E5A8F5B7428BE00039F500C755B5D
:1018990028755A00740D900050F0AE5AAF5B900055
:1018A9008CE012694B74288E048F05FF12693B8CFA
:1018B9005A8D5BAE28AF29740A8E048F05FF126911
:1018C9003B8D068C07AC5AAD5BCFCECF12000374AB
:1018D9000A8E048F05FF12693B8C5A8D5BAE28AFC7
:1018E90029EF2DFDEE3CFC8C288D29229000E7E0A4
:1018F900B4026AE55F75F00884FF7E008F37E55F03
:1019090075F00884ADF07C008D3A753F08755A0171
:10191900755BE0E537C3943F5005120D6A80069068
:101929000280E0F53785372D752C00AE2CAF2DAC34
:101939002AAD2B12000374648E048F05FF12693BD4
:101949008C2C8D2D900084E08C068D0712694B74C8
:10195900648E048F05FF12693B8C2C8D2DAE28AF48
:1019690029AC2AAD2B12000374648E048F05FF1273
:10197900693B8C288D29900084E08C068D071269BB
:101989004B74648E048F05FF12693B8C288D29A244
:101999000D401DAE52AF537405BE00039F5002D2D5
:1019A9000DE561D394CC4008D2017411900050F038
:1019B9009000E6E0B402089000D4E0640B60028075
:1019C90035AE28AF29E56B12694B74E78E048F0594
:1019D900FF12693B8C288D299000E7E0B40217AE0D
:1019E9002CAF2DE56B12694B74E78E048F05FF123E
:1019F900693B8C2C8D2D9000A6E05402601B900051
:101A09009DE0A852B80012D39553400DA20DB3B36F
:101A19005007E561C3949A40028028AE34AF3590EF
:101A2900009BE075F002A4FDACF0EF2DFDEE3CFC4F
:101A390074022DFD50010CE561BC0007D39D4003E4
:101A4900754301856135753400E5437003021B3820
:101A59009000F9E0C395435003021B2A900109E065
:101A6900C394025076E56775F00A84FF7E009005FD
:101A790081126972E0F55B755A00AE5AAF5B90004E
:101A89009CE012694B74648E048F05FF12693B8CCC
:101A99005C8D5D9000F9E004C395438C068D0712B7
:101AA900694B9000F9E08E048F05FF12693B8C5C4D
:101AB9008D5DAE28AF29EF2DFDEE3CFC8C288D29DC
:101AC9009000E7E0B40212AE2CAF2DAA5CAB5DEF3B
:101AD9002BFBEE3AFA8A2C8B2D80469000F9E00414
:101AE900C39543854BF0A4FFAEF09000F9E08E0456
:101AF9008F05FF12693B8C5C8D5DAE28AF29EF2DF8
:101B0900FDEE3CFC8C288D299000E7E0B40212AE72
:101B19002CAF2DAA5CAB5DEF2BFBEE3AFA8A2C8B2E
:101B29002D05439000F9E0C3954350037543009098
:101B390000A6E05401601B90009AE0A852B8001278
:101B4900D39553400DA20DB3B35007E55FC394CCB1
:101B590040028025900098E075F003A4FFAEF0E5FF
:101B6900402FFF50010E74032FFF50010EE55FBE99
:101B79000007D39F4003754401855F40E544700326
:101B8900021C6B9000FAE0C395445003021C5D905F
:101B99000109E0C394025076E56775F00A84FF7E77
:101BA90000900581126972E0F55B755A00AE5AAF73
:101BB9005B900099E012694B74648E048F05FF12E3
:101BC900693B8C5C8D5D9000FAE004C395448C06FA
:101BD9008D0712694B9000FAE08E048F05FF126998
:101BE9003B8C5C8D5DAE28AF29EF2DFDEE3CFC8C66
:101BF900288D299000E7E0B40212AE2CAF2DAA5C23
:101C0900AB5DEF2BFBEE3AFA8A2C8B2D80469000C8
:101C1900FAE004C39544854CF0A4FFAEF09000FAB5
:101C2900E08E048F05FF12693B8C5C8D5DAE28AF99
:101C390029EF2DFDEE3CFC8C288D299000E7E0B4BE
:101C49000212AE2CAF2DAA5CAB5DEF2BFBEE3AFA7C
:101C59008A2C8B2D05449000FAE0C39544500375F6
:101C690044009000FCE02529FFAE2850010E8E2883
:101C79008F299000ABE0A828B80004952950099055
:101C890000ABE0F5297528009000E7E0B4020D905B
:101C990000ABE0A82CB80006952D40028009900001
:101CA900ABE0F52D752C00229000E7E0B40102802D
:101CB90003021DBCA20DB35003021DBA9000B2E08D
:101CC900B40168AE28AF29AC52AD53120003743C7D
:101CD9008E048F05FF12693B9000C2E0BC00109D85
:101CE900400D9000C4E0A828B8000495295002D2FC
:101CF90002AE28AF29AC52AD53120003743C8E04D6
:101D09008F05FF12693B9000C2E0C3940ABC00151D
:101D1900D39D40119000C4E0C39405A828B80005DC
:101D2900D3952950028002C2028068AE28AF29AC3F
:101D390052AD5312000374788E048F05FF12693B6C
:101D49009000C2E0BC00109D400D9000C4E0A8289E
:101D5900B8000495295004D2028038AE28AF29ACC6
:101D690052AD5312000374788E048F05FF12693B3C
:101D79009000C2E0C3940ABC0015D39D40119000A5
:101D8900C4E0C39405A828B80005D395295002805A
:101D990002C202A202B34019AE28AF299000C3E0E3
:101DA90012694B74648E048F05FF12693B8C288D70
:101DB900298002C202A200B34006A201B3B35009AE
:101DC900900019E4F0A3F08024AE28AF297400D361
:101DD9009F74019E400C900019E528F0A3E529F0B5
:101DE900800B74FF900019F8E4F0E8A3F09000C9A3
:101DF900E0D39402400C9000B4E07006A20DB3B396
:101E09004002801AAE28AF29740212694B8E288FBE
:101E190029AE2CAF2D740212694B8E2C8F2D900098
:101E2900B2E0B4011AAE28AF29740212694B8E28A8
:101E39008F29AE2CAF2D740212694B8E2C8F2DAECB
:101E490028AF29745E12694B740A8E048F05FF123C
:101E5900693B8C288D299000E7E0B40217AE2CAFBE
:101E69002D745E12694B740A8E048F05FF12693B4B
:101E79008C2C8D2DAE28AF297402BE000AD39F4049
:101E890006752902752800AE2CAF2D7402BE000A12
:101E9900D39F4006752D02752C00900017E528F098
:101EA900A3E529F02290004FE090038112697DE0BB
:101EB900F54175426490004FE0FE9000BDE0D39E6D
:101EC9004037E55F75F00884FF7E008F37E55F7561
:101ED900F00884ADF07C008D3A753F08755A03759A
:101EE9005B96E537C3941F5005120D6A800690046E
:101EF90036E0F5378537428035E55F75F00884FFB0
:101F09007E008F37E55F75F00884ADF07C008D3A6F
:101F1900753F08755A03755BB6E537C3941F5005BD
:101F2900120D6A8006900456E0F5378537422290F3
:101F390000F3E0F53C753F11755A04755B00AE522C
:101F4900AF53E53C75F00FA4FDACF0EDD39FEC9ECB
:101F59004021E53C8E048F05FF12693BED75F010B9
:101F6900A4FFAEF0E55F75F01184FD7C00ED2FF55F
:101F79003D800EE55F75F01184FF7E00EF24F0F5DA
:101F89003D853D37E55F75F01184AFF07E008F3AEE
:101F9900120D6A85373EAE52AF539000F3E075F0EB
:101FA9000FA4FDACF0EDD39FEC9E4028755A047543
:101FB9005B10853D37120D6A853E38853739AE523B
:101FC900AF53E53C8E048F05FF1269668D3A853C57
:101FD9003B120DE4853741754264229000F3E0F528
:101FE9003C753F11755A04755B00AE52AF53E53C21
:101FF90075F00FA4FDACF0EDD39FEC9E4021E53CBC
:102009008E048F05FF12693BED75F010A4FFAEF049
:10201900E56175F01184FD7C00ED2FF53D800EE53D
:102029006175F01184FF7E00EF24F0F53D853D37A1
:10203900E56175F01184AFF07E008F3A120D6A8563
:10204900373EAE52AF539000F3E075F00FA4FDACEC
:10205900F0EDD39FEC9E4028755A04755B10853DC1
:1020690037120D6A853E38853739AE52AF53E53C94
:102079008E048F05FF1269668D3A853C3B120DE48B
:102089008537417542649000BCE0B4047990004FF3
:10209900E0FE9000BDE0D39E4037E55F75F008840F
:1020A900FF7E008F37E55F75F00884ADF07C008D09
:1020B9003A753F08755A03755B96E537C3941F5007
:1020C90005120D6A8006900436E0F537853742809F
:1020D90035E55F75F00884FF7E008F37E55F75F0A1
:1020E9000884ADF07C008D3A753F08755A03755B1D
:1020F900B6E537C3941F5005120D6A800690045641
:10210900E0F53785374222900087E0B4013BE56767
:1021190075F00A84FF7E008F37E56775F00A84AD94
:10212900F07C008D3A753F0A755A05755B12E537E3
:10213900C394115005120D6A80069005A4E0F53785
:10214900E5422537C39464F542900088E0B4013B29
:10215900E56875F00A84FF7E008F37E56875F00A37
:1021690084ADF07C008D3A753F0A755A05755B7E22
:10217900E537C394115005120D6A8006900610E0E8
:10218900F537E5422537C39464F542E5412542F523
:102199003690008FE0B402109007CBE02536FE9010
:1021A90000E3E0F4042EF5369000E6E0D394014014
:1021B90040E56BC394E7501D74E7C3956BFE900728
:1021C900CDE08E00F5F0E884FF7E008F37E53625F7
:1021D90037F536801CE56BC394E7FE9007CDE08E9A
:1021E90000F5F0E884FF7E008F37E536C39537F5B3
:1021F90036A20D4006E5412464F536E536D39464EC
:102209004009E536C39464F53680037536009000BD
:10221900BFE0C3953650069000BFE0F53622D200E4
:10222900900079E0A852B800049553504190007984
:10223900E0A852B800049553500375360F90007901
:10224900E004A852B800049553500375360A90006B
:1022590079E02402A852B800049553500575360553
:10226900C200900079E060067409900050F0C23C09
:102279007E017F009000C5E012694B9000D4E08E8A
:10228900048F05FF12693BE55FBC0017D39D40131E
:102299009000CEE0B40204D23C8002C200740A90DD
:1022A9000050F09000C6E0C3956750159000D8E043
:1022B900A852B8000495535002C200740B90005004
:1022C900F0E567C39464501D90011EE0600D900114
:1022D9001EE0A852B80006955340028008C2007457
:1022E9000B900050F0A2004003753605900107E0FD
:1022F900B40114900108E0A852B80004955350079E
:10230900E55FC39560400280089000B0E0F5368033
:102319003A90008FE0B40306A22CB3B34002802B9D
:102329009007CFE0C39405A852B800049553500C08
:102339009000B0E0F536740C900050F09007CFE0B3
:10234900A852B8000495535002C20085366C90001B
:1023590081E02536FE90004FE075F01E84FC7F0079
:10236900EE2CF5362290004FE075F00584FF7E00D3
:102379008F3790004FE075F00584ADF07C008D3A01
:10238900753F05755A03755BD69000D2E01475F058
:102399000584FF7E00E537BE00039F5005120D6AD4
:1023A900800BE53790045712697DE0F537E53790E2
:1023B90007CEF09007CEE0FE9000C1E0C39E500822
:1023C9009000C1E09007CEF022E56775F00A84FF1E
:1023D9007E00900581126972E0F546E546D3946462
:1023E9004010E546C3946475F00F84FF7E008F4664
:1023F90080037546009000A4E02546F5462290002A
:10240900BCE0C3940350269007BBE0FEA3E0FF7431
:1024190004120039E55F12694B740F8E048F05FFB2
:1024290012693B9007B9ECF0A3EDF080249007BB4B
:10243900E0FEA3E0FF7404120039E56112694B74F0
:102449000F8E048F05FF12693B9007B9ECF0A3EDDD
:10245900F0900097E0B40262E56AC3944175F00513
:1024690084FF7E008F37E56A75F00584ADF07C0046
:102479008D3A753F05755A06755B14E537C3941790
:102489005005120D6A80069006A8E0F5379007B945
:10249900E0FEA3E0FF740A8E048F05FF12693BE595
:1024A900378C068D0712694B740A8E048F05FF124B
:1024B900693B9007B9ECF0A3EDF09007B9E0FEA3F2
:1024C900E0FF9007BFE0FCA3E0FDEDD39FEC9E4049
:1024D9000F9007BFE0F8A3E09007B9C8F0A3C8F0D0
:1024E900229006C8E090386BF8282873804C8553F1
:1024F9007380479000D4E0855FF0A4FFAEF07408C4
:102509001200398F738033856173802E85677380DC
:10251900298568738024856973801F856A73801A89
:10252900856B7380158566738010856573800B854F
:0A2539006C73800690001AE0F57341
:10386B000224F50224F70224FC022510022515027E
:10387B00251A02251F02252402252902252E0225A1
:07388B003302253802253D40
:102543009006C9E0FE9006CAE0D39E404B9006C8B1
:10255300E0B404189006CAE0C395735002D22D90DC
:1025630006C9E0D395734002C22D802A9006C9E0C4
:10257300C3957350099006CAE0D395735002800245
:10258300D22D9006C9E0D3957350099006CAE0C3D3
:1025930095735002C22D802A9006C9E0D3957340EB
:1025A300099006CAE0C3957340028002C22D9006CB
:1025B300C9E0C3957340099006CAE0D395734002FE
:1025C300D22D229006CCE0903892F8282873804CC4
:1025D30085537380479000D4E0855FF0A4FFAEF08D
:1025E30074081200398F738033856173802E856779
:1025F3007380298568738024856973801F856A7356
:10260300801A856B7380158566738010856573806A
:0C2613000B856C73800690001AE0F573D4
:103892000225D10225D30225D80225EC0225F10208
:1038A20025F60225FB02260002260502260A02262A
:0738B2000F02261402261983
:10261F009006CDE0FE9006CEE0D39E405F9006CCB4
:10262F00E0B404189006CEE0C395735002D22E90FA
:10263F0006CDE0D395734002C22E803E9006CDE0CA
:10264F00C3957350099006CEE0D395735002800264
:10265F00D22E9006CDE0D3957350099006CEE0C3ED
:10266F0095735002C22E9006CCE0B401099000E0A1
:10267F00E0D3956150028002C22E802A9006CDE0F1
:10268F00D3957340099006CEE0C395734002800244
:10269F00C22E9006CDE0C3957340099006CEE0D3CD
:1026AF0095734002D22E229006D0E09038B9F828C8
:1026BF002873804C85537380479000D4E0855FF07A
:1026CF00A4FFAEF074081200398F738033856173E5
:1026DF00802E856773802985687380248569738050
:1026EF001F856A73801A856B7380158566738010DA
:1026FF00856573800B856C73800690001AE0F57307
:1038B9000226C10226C30226C80226DC0226E1022C
:1038C90026E60226EB0226F00226F50226FA022651
:0738D900FF0227040227098A
:10270F009006D1E0FE9006D2E0D39E404B9006D0CB
:10271F00E0B404189006D2E0C395735002D22F9004
:10272F0006D1E0D395734002C22F802A9006D1E0E4
:10273F00C3957350099006D2E0D39573500280026F
:10274F00D22F9006D1E0D3957350099006D2E0C3F3
:10275F0095735002C22F802A9006D1E0D395734013
:10276F00099006D2E0C3957340028002C22F9006F3
:10277F00D1E0C3957340099006D2E0D39573400220
:10278F00D22F229006D4E09038E0F8282873804C9E
:10279F0085537380479000D4E0855FF0A4FFAEF0BF
:1027AF0074081200398F738033856173802E8567AB
:1027BF007380298568738024856973801F856A7388
:1027CF00801A856B7380158566738010856573809D
:0C27DF000B856C73800690001AE0F57307
:1038E00002279D02279F0227A40227B80227BD02B4
:1038F00027C20227C70227CC0227D10227D60227D8
:07390000DB0227E00227E5CE
:1027EB009006D5E0FE9006D6E0D39E404B9006D4E3
:1027FB00E0B404189006D6E0C395735002D2309023
:10280B0006D5E0D395734002C230802A9006D5E0FE
:10281B00C3957350099006D6E0D39573500280028E
:10282B00D2309006D5E0D3957350099006D6E0C30D
:10283B0095735002C230802A9006D5E0D395734031
:10284B00099006D6E0C3957340028002C230900611
:10285B00D5E0C3957340099006D6E0D3957340023B
:10286B00D230229006D8E0903907F8282873804C94
:10287B0085537380479000D4E0855FF0A4FFAEF0E2
:10288B0074081200398F738033856173802E8567CE
:10289B007380298568738024856973801F856A73AB
:1028AB00801A856B738015856673801085657380C0
:0C28BB000B856C73800690001AE0F5732A
:1039070002287902287B022880022894022899023B
:10391700289E0228A30228A80228AD0228B202285E
:07392700B70228BC0228C111
:1028C7009006D9E0FE9006DAE0D39E404B9006D8FA
:1028D700E0B404189006DAE0C395735002D2319041
:1028E70006D9E0D395734002C231802A9006D9E019
:1028F700C3957350099006DAE0D3957350028002AE
:10290700D2319006D9E0D3957350099006DAE0C327
:1029170095735002C231802A9006D9E0D39573404F
:10292700099006DAE0C3957340028002C23190062F
:10293700D9E0C3957340099006DAE0D39573400256
:10294700D231229006DCE090392EF8282873804C8B
:1029570085537380479000D4E0855FF0A4FFAEF005
:1029670074081200398F738033856173802E8567F1
:102977007380298568738024856973801F856A73CE
:10298700801A856B738015856673801085657380E3
:0C2997000B856C73800690001AE0F5734D
:10392E0002295502295702295C02297002297502C3
:10393E00297A02297F02298402298902298E0229E5
:07394E009302299802299D54
:1029A3009006DDE0FE9006DEE0D39E404B9006DC11
:1029B300E0B404189006DEE0C395735002D232905F
:1029C30006DDE0D395734002C232802A9006DDE033
:1029D300C3957350099006DEE0D3957350028002CD
:1029E300D2329006DDE0D3957350099006DEE0C342
:1029F30095735002C232802A9006DDE0D39573406E
:102A0300099006DEE0C3957340028002C23290064D
:102A1300DDE0C3957340099006DEE0D39573400271
:102A2300D232229006E0E0903955F8282873804C82
:102A330085537380479000D4E0855FF0A4FFAEF028
:102A430074081200398F738033856173802E856714
:102A53007380298568738024856973801F856A73F1
:102A6300801A856B73801585667380108565738006
:0C2A73000B856C73800690001AE0F57370
:10395500022A31022A33022A38022A4C022A51024B
:103965002A56022A5B022A60022A65022A6A022A6C
:073975006F022A74022A7997
:102A7F009006E1E0FE9006E2E0D39E404B9006E028
:102A8F00E0B404189006E2E0C395735002D233907D
:102A9F0006E1E0D395734002C233802A9006E1E04D
:102AAF00C3957350099006E2E0D3957350028002EC
:102ABF00D2339006E1E0D3957350099006E2E0C35C
:102ACF0095735002C233802A9006E1E0D39573408C
:102ADF00099006E2E0C3957340028002C23390066C
:102AEF00E1E0C3957340099006E2E0D3957340028D
:102AFF00D233229006E4E090397CF8282873804C7A
:102B0F0085537380479000D4E0855FF0A4FFAEF04B
:102B1F0074081200398F738033856173802E856737
:102B2F007380298568738024856973801F856A7314
:102B3F00801A856B73801585667380108565738029
:0C2B4F000B856C73800690001AE0F57393
:10397C00022B0D022B0F022B14022B28022B2D02D3
:10398C002B32022B37022B3C022B41022B46022BF3
:07399C004B022B50022B55DA
:102B5B009006E5E0FE9006E6E0D39E404B9006E43F
:102B6B00E0B404189006E6E0C395735002D234909B
:102B7B0006E5E0D395734002C234802A9006E5E067
:102B8B00C3957350099006E6E0D39573500280020B
:102B9B00D2349006E5E0D3957350099006E6E0C376
:102BAB0095735002C234802A9006E5E0D3957340AA
:102BBB00099006E6E0C3957340028002C23490068A
:102BCB00E5E0C3957340099006E6E0D395734002A8
:102BDB00D234229006E8E09039A3F8282873804C71
:102BEB0085537380479000D4E0855FF0A4FFAEF06F
:102BFB0074081200398F738033856173802E85675B
:102C0B007380298568738024856973801F856A7337
:102C1B00801A856B7380158566738010856573804C
:0C2C2B000B856C73800690001AE0F573B6
:1039A300022BE9022BEB022BF0022C04022C09025E
:1039B3002C0E022C13022C18022C1D022C22022C7A
:0739C30027022C2C022C311D
:102C37009006E9E0FE9006EAE0D39E404B9006E856
:102C4700E0B404189006EAE0C395735002D23590B9
:102C570006E9E0D395734002C235802A9006E9E081
:102C6700C3957350099006EAE0D39573500280022A
:102C7700D2359006E9E0D3957350099006EAE0C390
:102C870095735002C235802A9006E9E0D3957340C8
:102C9700099006EAE0C3957340028002C2359006A8
:102CA700E9E0C3957340099006EAE0D395734002C3
:102CB700D235229006ECE09039CAF8282873804C68
:102CC70085537380479000D4E0855FF0A4FFAEF092
:102CD70074081200398F738033856173802E85677E
:102CE7007380298568738024856973801F856A735B
:102CF700801A856B73801585667380108565738070
:0C2D07000B856C73800690001AE0F573D9
:1039CA00022CC5022CC7022CCC022CE0022CE502E8
:1039DA002CEA022CEF022CF4022CF9022CFE022D06
:0739EA0003022D08022D0D60
:102D13009006EDE0FE9006EEE0D39E404B9006EC6D
:102D2300E0B404189006EEE0C395735002D23690D7
:102D330006EDE0D395734002C236802A9006EDE09B
:102D4300C3957350099006EEE0D395735002800249
:102D5300D2369006EDE0D3957350099006EEE0C3AA
:102D630095735002C236802A9006EDE0D3957340E6
:102D7300099006EEE0C3957340028002C2369006C6
:102D8300EDE0C3957340099006EEE0D395734002DE
:102D9300D23622AE2EAF2F74F5D39F74019E400816
:102DA300782E12699F022EB0752F01752E00AE5238
:102DB300AF53E546BE000DD39F40099000B6E0D364
:102DC300954740028023754700E546C39553F57345
:102DD3009000B9E0D395454008E5452573F5458056
:102DE300069000B9E0F54580020547900092E0D3D4
:102DF3009561401CE55FC395604015AE52AF53E546
:102E030046BE00039F50099000B7E0D395484002A7
:102E1300806E9007D2E0A852B80004955350037512
:102E23004A009007D2E0A852B8000BD3955340064E
:102E3300E5539007D2F0E54A7041E553C39546F553
:102E430073E573D3940540037573059000B8E0C32D
:102E530095455007E573C3954540028009E545C391
:102E63009573F54580069000B8E0F5459000B8E00D
:102E7300D3954540069000B8E0F5457548008002BB
:102E83000548E54A7016900092E0C39561500DE540
:102E9300462405A852B8000695534002800F9000BF
:102EA300A5E0F545754A0174789007D2F022AE2E5D
:102EB300AF2F74E9D39F74039E4008782E12699F45
:102EC30002304F752F01752E00754532A237402A07
:102ED3007545199000A5E075F002A4FFAEF0E54733
:102EE300BE0006D39F4002D2370547754A03747864
:102EF3009007D2F075490002303EAE52AF53E5461B
:102F03006F4E700302303EE546BE000DD39F40096D
:102F13009000B6E0D395474002800F754700E54A1D
:102F2300C394035003754519800DE546C39553F5C6
:102F330073E5472573F547900092E0D39561400E02
:102F43009007D2E0A852B80007D395534002800CF3
:102F530005499000A5E0B54903754A00E54AB40365
:102F630006A20DB3B34002800A0549E549B43C0308
:102F7300754A02E54AB402299007D2E0A852B80084
:102F83000ED395534009E5539007D2F0754900904D
:102F93000092E0C39561500975490074789007D297
:102FA300F0E54A705A900092E0D39561401CE55FCA
:102FB300C395604015AE52AF53E546BE00039F5024
:102FC300099000B7E0D39548400280087548007522
:102FD300454B8028E553C39546F573E573D39405B4
:102FE3004003757305900092E0D395614008E5486E
:102FF3002573F5488006E5482406F548754900E53C
:103003004A7016900092E0C39561500DE546240581
:10301300A852B80006955340028003754A01E54A59
:10302300B4011875451905499000A5E0B549067521
:103033004A0275490074789007D2F0E54575F00AA5
:10304300A4FFAEF09007C3EEF0A3EFF022E56F907C
:1030530039F1F828287390008AE0700302327790E0
:1030630000C0E0B40102800302319290004DE0B54C
:103073005E02800302318F7E017F00E5BE12694B41
:10308300E5BD2FFF50010E8E5A8F5B741012694BF2
:10309300900078E08E048F05FF12693B9007C7EC20
:1030A300F0A3EDF074FFBC00039D500B74FF900779
:1030B300C7F8E4F0E8A3F0E56B600FE56BC394FE9B
:1030C30050089000E6E06402600280649000D4E05F
:1030D300B40B1F9007C7E0FEA3E0FF74E712694B30
:1030E300E56B8E048F05FF12693B9007C7ECF0A3D5
:1030F300EDF09000D4E0D3940B40089000BCE06462
:10310300046002802B9007C7E0FEA3E0FF9007C98D
:10311300E0FCA3E0FDEFD39DEE9C400D1269979078
:1031230007C7EEF0A3EFF080079007C7E4F0A3F022
:1031330090008AE0B4021E9007C7E0FEA3E0FF9070
:1031430007D3E02FFF50010E74011200399007C717
:10315300EEF0A3EFF09007C7E0FEA3E0FF9007D3E4
:10316300E0BE0008D39F4004D23A8002B23A9007EF
:10317300C8E09007D3F09000BCE064016006A23A77
:10318300B3B3400280069007C8E0F55F023275D200
:103193003A7E017F00E5BE12694BE5BD2FFF50016A
:1031A3000E8E5A8F5B741012694B900078E08E0478
:1031B3008F05FF12693B9007C7ECF0A3EDF0E56BB9
:1031C300600FE56BC394FE50089000E6E064026074
:1031D3000280649000D4E0B40B1F9007C7E0FEA305
:1031E300E0FF74E712694BE56B8E048F05FF1269EC
:1031F3003B9007C7ECF0A3EDF09000D4E0D3940B21
:1032030040089000BCE064046002802B9007C7E094
:10321300FEA3E0FF9007C9E0FCA3E0FDEFD39DEE22
:103223009C400D1269979007C7EEF0A3EFF080075B
:103233009007C7E4F0A3F090008AE0B4021E900761
:10324300C7E0FEA3E0FF9007D3E02FFF50010E7409
:10325300011200399007C7EEF0A3EFF09007C8E022
:103263009007D3F09000BCE0640160069007C8E0CB
:10327300F55F8003755F00900086E07006756F014F
:1032830002305075BB18023845900086E070030287
:1032930033FD7E017F00E5BE12694BE5BD2FFF5074
:1032A300010E8E5A8F5B9000CCE0B4010F7E0F7F2E
:1032B300FFAC5AAD5B1269978E5A8F5B9000F1E0B9
:1032C300B40245AE5AAF5B900023E0FCA3E0FDEDF2
:1032D300D39FEC9E400A900023E55AF0A3E55BF0F0
:1032E300AE5AAF5B900025E0FCA3E0FDEFD39DEE6B
:1032F3009C400A900025E55AF0A3E55BF0AE5AAF77
:103303005B74041200398F619000F1E0704CAE5A87
:10331300AF5B900023E0FCA3E0FDEFD39DEE9C4068
:10332300091269978E5A8F5B8006755B00755A0088
:10333300AE5AAF5B741012694B900075E08E048F28
:1033430005FF12693B8C5A8D5B74FFBC0009D39D4A
:103353004005855B6180037561FE9000BCE0B401AC
:103363000280030233FBA20DB3B3500E900090E032
:10337300A852B80005D39553500280719000CDE058
:103383008561F0A4FFAEF074648E048F05FF1269AB
:103393003B8C5A8D5BE56B6016E56BC394FE500F57
:1033A3009000E6E0B402089000D4E0640B60028071
:1033B30017AE5AAF5B74E712694BE56B8E048F054A
:1033C300FF12693B8C5A8D5BAE5AAF5B9007C7E027
:1033D300FCA3E0FDEDD39FEC9E4005855B5F800B76
:1033E300A23AB340069007C8E0F55F800BA23AB358
:1033F30040069007C8E0F55F80037561009000897F
:10340300E07006756F0202305075BB1902384590A3
:103413000089E070030234B2E55ED39551400302A4
:1034230034B0900021E0FEA3E0FFE56512698F90C0
:103433000021EEF0A3EFF07E017F00E5BE12694BA1
:10344300E5BD2FFF50010E8E5A8F5B9000F6E070A2
:1034530013740A12694B74518E048F05FF12693B72
:103463008D658019AE5AAF5B740A12694B8F048E57
:10347300057E017F95CDCCCD1268398F65E565D387
:1034830094644003756564900021E0FEA3E0FFE5CA
:10349300652FFF50010E900021EEF0A3EFF0900096
:1034A3008DE0048E048F05FF12693B8D65800375E3
:1034B30065329000D9E07006756F0302305075BB1A
:1034C300130238459000D9E0604A7E017F00E5BED3
:1034D30012694BE5BD2FFF50010E8E5A8F5B7404AA
:1034E3001200398F669000DBE08566F0A4FDACF036
:1034F3007464FF12693B8D669000DAE08566F0A480
:10350300FFAEF074FF8E048F05FF12693BED900050
:1035130074F08003756600900087E07006756F0491
:1035230002305075BB17023845900087E0B40102A2
:1035330080030235C07E017F00E5BE12694BE5BD05
:103543002FFF50010E8E5A8F5B9007D4E0601990C5
:1035530007D4E0149063C512008CE493FC740193C8
:10356300FDEDC39FEC9E400280069007D4E014F06B
:103573009007D4E0C394B3501DAE5AAF5B9007D409
:10358300E0049063C512008CE493FC740193FDEF97
:10359300C39DEE9C400280069007D4E004F09007A0
:1035A300D4E0FE9000ADE08E0088F0A4FFAEF0748E
:1035B300648E048F05FF12693B8D67800375670076
:1035C300900088E07006756F0502305075BB1602D7
:1035D3003845900088E0B4010280030236697E0119
:1035E3007F00E5BE12694BE5BD2FFF50010E8E5AD9
:1035F3008F5B9007D5E060199007D5E01490652F95
:1036030012008CE493FC740193FDEDC39FEC9E4088
:103613000280069007D5E014F09007D5E0C394B379
:10362300501DAE5AAF5B9007D5E00490652F120092
:103633008CE493FC740193FDEFC39DEE9C400280E8
:10364300069007D5E004F09007D5E0FE9000B3E0C4
:103653008E0088F0A4FFAEF074648E048F05FF1211
:10366300693B8D68800375680075BB1F0238457E12
:10367300017F00E5BE12694BE5BD2FFF50010E8EA1
:103683005A8F5B740912694B74E68E048F05FF121F
:10369300693B8D6A90008FE07006756F07023050AA
:1036A30075BB1502384590008FE070030237C47E66
:1036B300017F00E5BE12694BE5BD2FFF50010E8E61
:1036C3005A8F5B74041200398F6990008FE0B40144
:1036D300159000E3E08569F0A4FFAEF074071200D3
:1036E30039EF9007CCF090008FE0B402159000E31F
:1036F300E08569F0A4FFAEF07407120039EF90077C
:10370300CBF090008FE0B4030280030237A7900050
:10371300D0E0701CE569C394195002D22CE569D33B
:1037230094644002C22C9000AFE09007CFF0806316
:103733009000AFE070349000E3E08569F0A4FFAE41
:10374300F074FF8E048F05FF12693BED9007CFF0F5
:10375300AE52AF53741EBE0006D39F4002D22CE577
:1037630061D394E54002C22C8029E569C3940A50D1
:103773000DAE52AF53741EBE0004D39F500280029D
:10378300D22CE561D394E54002C22C9000AFE090C7
:1037930007CFF09007CFE0C3940550067405900758
:1037A300CFF0C23B90008FE0B40414E569C39419D1
:1037B3005002D23BE569D394324002C23BC22C8013
:1037C300037569009000E6E07006756F08023050DB
:1037D30075BB14806D9000E6E060567E017F00E5C6
:1037E300BE12694BE5BD2FFF50010E8E5A8F5BEF62
:1037F300D39421EE940E4005756BFF8015AE5AAF3E
:103803005B741012694B74E38E048F05FF12693BDE
:103813008D6BE56B75F00BA4FFAEF09000D4E08EDA
:10382300048F05FF12693B9007C9ECF0A3EDF0800C
:1038330003756B0090008AE0600575BB1A80037501
:02384300BB18B0
:1039F10002305902328C0234120234C702352C02D1
:0B3A010035D50236720236A90237D814
:05384500056FD2EC222A
:09697D002582F5825002058322F7
:0F008C0025E050020583258250020583F582226C
:10691A00EF2F500205832582F582E5833E2EF5830B
:01692A00224A
:10698F00CFC39FFF50011E22C3EF9DFFEE9CFE223F
:08699F000806B60002180622EA
:0D695900A3E004F07006120049E004F022F3
:0E003900048007C3CE13CECF13CFD5E0F6223E
:10683900BC000FBE0008ED8FF084FFADF022E4FE2E
:10684900FF22BE000DEF60FE54F0606F20E70302E7
:1068590068EFEAC0E0EBC0E078017A0075F001EE7C
:1068690020E710EF25E0FFEE33FE0AC5F023C5F05F
:1068790030E7F0EA5407F9096A7A007B00600108F9
:10688900C3EC9E40167004ED9F4010ED9FFDEC9EF9
:10689900FCE5F0CA4ACA03F5F08005E5F003F5F016
:1068A900C3EE13FEEF13FFD9D77908CACBCAD8D0E4
:1068B900EAFEEBFFD0E0FBD0E0FA22EC8FF084FC9B
:1068C900ED54F045F0C48FF084FEEDC454F045F06A
:1068D900C48FF084FDEEC4FE54F02DFFEE540F3C3E
:1068E900FEADF07C0022790078008FF0EC7E082064
:1068F900E70DC3CD33CD33C933C9C833C8DEF084FE
:1069090049F9E5F08FF0BE00E6FD7C00E9FFE8FEFD
:01691900225B
:0E694B00F88FF0A4FFE5F0CE88F0A42EFE2217
:10000300EF8DF0A4F9A8F0EF8CF0A428F8EE8DF0B2
:06001300A428FEE9FF2213
:10692B00600D782B026935007830D8FED5E0F8225F
:10693B00EEC0E07E00126839EFFDEEFCD0E0FE22E7
:0C696600EEC0E07E00126839D0E0FE2296
:03001B0002001EC2
:0300530002005652
:03009B00020071EF
:030000000269860C
:0969860075817575D00002444EC4
:0B697200E5822FF582E5833EF58322CD
:0A0049000582D5820215831582227C
:10001E00C0E0C0F0C083C082C0D075D0001243BA19
:0B002E00D0D0D082D083D0F0D0E032E0
:10005600C0E0C0F0C083C082C0D075D0001243BDDE
:10006600D0D0D082D083D0F0D0E032C0E0C0F0C093
:1000760083C082C0D075D0001243D9D0D0D082D0F0
:0600860083D0F0D0E0324F
:00000001FF
